:020000040800F2
:10400000783C002045F60008A9F30008ABF300084F
:10401000ADF30008AFF30008B1F3000800000000A2
:10402000000000000000000000000000B3F30008E2
:10403000B5F3000800000000B7F30008B9F300086A
:10404000A5F70008A9F70008ADF70008B1F70008C8
:10405000B5F70008B9F70008BDF70008C1F7000878
:10406000C5F70008C9F70008CDF70008D1F7000828
:10407000D5F70008D9F70008DDF70008E1F70008D8
:10408000E5F70008E9F70008E9770008F1F700080C
:10409000BBF30008F9F70008FDF70008C7F30008B4
:1040A00005F8000809F800080DF8000811F80008E4
:1040B000BFF30008C3F300081DF8000821F800084A
:1040C00025F8000829F800082DF8000831F8000844
:1040D00035F8000839F800083DF8000841F80008F4
:1040E00045F8000849F800084DF8000851F80008A4
:1040F00055F8000859F800085DF8000861F8000854
:1041000065F8000869F800086DF8000871F8000803
:1041100075F8000879F800087DF8000881F80008B3
:1041200085F8000889F800088DF8000891F8000863
:104130000A225143002807D101EBC101052091FB60
:10414000F0F101F5486106E001EB8101A1F57A513A
:10415000092091FBF0F1104691FBF0F002FB1012E8
:10416000052A02DB401C00B2704700B2704770B5F0
:10417000DFF8D44A00206060606101F07EFC0A250F
:10418000DFF8C86AF16A6943814206D20420DFF889
:10419000C01A0870082001F045FB012001F042FB25
:1041A000F0694543256170BD80B501F0D2FA04285D
:1041B00009D100BF14A0009008231A4611464420DC
:1041C00002F019FC01BD01F0C4FA022803D001F08D
:1041D000C0FA012809D100BF0DA0009008231A469B
:1041E0001146442002F007FC01BD01F0B2FA052897
:1041F00008D100BF08A0009008231A4611464420A9
:1042000002F0F9FB01BD0000FFFF81EDEDF3FFFFC0
:10421000FFC3BDBD9D83BFFFFFFF81BDBDDBE7FFCA
:1042200018B585B0002819D0DFF8284A01F025FC20
:104230002080208802F096FDDFF81C1A02F0A0FD15
:1042400002F01CFE02460B460BA1684602F03AFE45
:104250006A460021422000F0ABFC0BE001F00DFCAF
:10426000024664A1684602F07CFE002269461046C0
:1042700000F0F3FB06B010BD252E31663A3B00007E
:10428000401E072815D8DFE800F00406080A0C0EC7
:10429000101280207047C0207047E0207047F02047
:1042A0007047F8207047FC207047FE207047FF20C1
:1042B000704700207047000030B585B001F0DDFB8D
:1042C00002F050FD044601F0D8FB02F04BFD214600
:1042D00002F0DEFE044602F047FF0546DFF87C09E7
:1042E000006802F03FFD0146204602F049FD2946E4
:1042F00002F0CEFE03F0FAFADFF86419088080B20B
:1043000002F030FDDFF8501902F03AFD02F0B6FD80
:1043100002460B4605A1684602F0D4FD6A4600211C
:10432000422000F045FC05B030BD0000252E31666E
:104330003C3B00007FB502F017FF4FF0834102F0D5
:10434000A7FE03F0D3FA0446E4B200252A4608216A
:1043500002A803F0FDFA112C24DA082C07DBFF2653
:10436000A4F10800C0B2FFF78BFF054603E020462A
:10437000FFF786FF064656EA050000D1802600209A
:1043800004E002A90D5401440E71401C0428F8DB1E
:104390000420019002A800901023042200213B2059
:1043A00002F061FB7FBD1CB504460A469BA168462E
:1043B00002F0D7FD684603F0EDFA0146DFF88C08FD
:1043C000806A002801D1432000E045206A460B4660
:1043D0009BB2D054491C202301E01354491C0846C9
:1043E00080B20428F9DB002111546946204600F010
:1043F000FBFA13BD2566560010B4014600200246A4
:104400000EE0E41FE34008E0012393400B4054001A
:10441000042AF6DAC4F10704A340DBB21818521CD0
:10442000072AF1DDC0B210BC70472DE9F84F98465D
:10443000DFF8C05B05F5D076002B12D1DFF8B84B62
:104440002378002B08D10023B361F361012323708B
:1044500000236370A3701DE03368B361F368F361F8
:1044600018E0012B12D1DFF8904B6378002B08D1B4
:104470000023B361F3612370012363700023A370F1
:1044800008E07368B3613369F36103E0B368B36153
:104490007369F3614FF0000982468B46144609E0C8
:1044A0001AF80900FFF7A8FFDFF8581B01F8090008
:1044B00009F1010921465F464F43B9EB470FEFD39E
:1044C000002301E003EB4103B3EB470F39D2002295
:1044D00016E02AFA00FA25F81CA007E0F069002887
:1044E000F7D1B0690AFA00FA25F81CA035F81C00CB
:1044F00082464FEA1A2A0EF80CA00EF80900521C48
:10450000A1464A45DED203EB020CE144DFF8F4EAAF
:104510001EF80C001EF809A04AEA002A25F81CA083
:1045200040460128DAD1B069002805D1F0690AFABD
:1045300000FA25F81CA0D9E72AFA00FA25F81CA0F1
:10454000D4E70024DFF8BC5A04E0285DFFF754FFED
:104550002855641CB4EB470FF7D3F069002806D147
:10456000B069102803D10020B0611020F061F0691B
:10457000002803D1B069401CB06101E0401EF06129
:10458000B069F1694246002A02D1F160306007E06B
:10459000B8F1010F02D17060316101E0B06071616A
:1045A000BDE8F18F1CB5DFF8844A207800280AD1D5
:1045B000DFF87C0A0090102360220021084602F0F8
:1045C0001AFA606021E0012809D160680090102388
:1045D00060220021084602F00EFA606015E0022811
:1045E00009D1DFF84C0A0090102360220021084610
:1045F00002F001FA09E0032807D160680090102357
:1046000060220021084602F0F6F92078401C207054
:10461000C0B2042801D10020207013BD2564000021
:10462000F8B582781646303E0A2E02D2A2F1300545
:10463000EDB2C2781646303E0A2E02D2A2F1300404
:10464000E4B200780246303A0A2A02D2A0F13003DE
:10465000DBB2002619E0DFF8D47BDFF8D40B182298
:1046600002FB036C10F80CC007EB060E8EF860C05E
:104670003744903702FB056C10F80CC087F800C077
:1046800002FB0462805C3876761C182EE3DB002780
:104690000C460FE0009610230C220021284600EB68
:1046A0004006B000C0B202F0A6F906466D1C082D07
:1046B000F0DB7F1C102F0CDADFF8706B200006D1C6
:1046C00002230C2208213046FFF7AFFED836002522
:1046D000EDE7002C09D14FF47A7002F064FD02F08E
:1046E0004CFABDE8F14003F0B1BCF1BD2DE9FF414A
:1046F00002460E46B5A7394601A802F032FC01A8D1
:1047000003F048F90146DFF84445A06A002801D1CA
:10471000432000E0452001AD0A4692B2A854491C4E
:10472000202201E02A54491C084680B20328F9DB04
:104730000021295401A9002000F056FADFF8F48A7C
:1047400098F80000411C88F80010DFF8FC1B01EB12
:104750004010009010231A460021292002F04BF946
:1047600098F80000032802D1002088F800003246A3
:10477000394601A802F0F5FB01A803F00BF9014648
:10478000A06A002801D1432000E045200A4692B2E9
:10479000A854491C202201E02A54491C084680B232
:1047A0000328F9DD0021295401A9382000F01CFA62
:1047B000BDE8FF817CB503F02CF9801E03280ED8DC
:1047C000DFE800F00205080BDFF8804B07E0DFF8B8
:1047D000804B04E0DFF87C4B01E0DFF87C4BDFF836
:1047E0007C0B009010231A460021084602F003F9C2
:1047F000022510E005EB850004EB800028380090CE
:1048000010230A220021284600EB80067000C0B267
:1048100002F0F1F86D1C092DECDB4FF4FA7002F098
:10482000C2FC50211020BDE87C4002F056B9F0B522
:10483000DFF8C467B17800290AD10121F1700021A5
:1048400031710821B1710021317071700121B17095
:10485000F17800292BD100237371DFF8A85713E0FA
:104860001C4600EB070CA4449CF833C005F804C0B8
:10487000944600EB0C0EA644774497F83370A4449A
:1048800005F80C705B1C737137797379B4799C42AD
:10489000E6D2641CB4717B1E3371E4B20B2C06D1DA
:1048A0000A20B071002030710120F070F0BD337922
:1048B000002B27D10123737113E01F468C46BC44A3
:1048C000DFF8404700F13305ED5D04F80C50154664
:1048D00000EB050E774497F83370654467555B1C11
:1048E0007371B4797379A342E7D3601EB071491C28
:1048F000F170C0B2002805D10120B07109203071DB
:104900000020F070F0BD00007CB504460D46DFF8D5
:10491000F46600221421304603F01AF8002C07D167
:1049200000230A220121DFF8F80BFFF77EFD11E0DA
:10493000012C07D101230A221946DFF8E80BFFF703
:1049400074FD07E0022C05D10A220121DFF8D00B0B
:10495000FFF76DFF00960A231A460621562002F043
:104960004AF800F05BFF042809D100BF1BA00090AB
:104970000A2306221146502002F03DF814E0002DD3
:1049800009D1DFF8A40B00900A230622114650201B
:1049900002F031F808E000BF0DA000900A230622C3
:1049A0001146502002F027F8FFF7FEFBA748406BA6
:1049B000002803D10120FFF733FC03E0012801D1D7
:1049C000FFF77AFCBDE87340B4E400002564000002
:1049D00000F0FEFFF000007F7F7F7F00FF0FE1E02F
:1049E0000FFFFF80BFBF80FFFEB504460D462401C8
:1049F0001CE00A2001E0363810263746FFB2C7F126
:104A0000100110220192DFF8242BC0B201EBD1710A
:104A1000491001EB40115018009010233246D2B2D9
:104A200000212046C0B202F01EF83C192878002868
:104A300012D015F8010B2028DBD02D2801D10C2035
:104A4000DBE7A0F130010A2902D230380E26D4E784
:104A5000A0F141010629CED3F7BD38B504460D4675
:104A6000002A27D12878002827D015F8010B2038F4
:104A7000DFF86C1CC0B201EB00100090102308227C
:104A80000021E000C0B201F0B6FF641CEAE715F8AF
:104A9000010B3038DFF8481CC0B201EB001000F504
:104AA000BE600090102308220021E000C0B201F097
:104AB000A2FF641C28780028E9D131BD1CB502464C
:104AC000DFF8204C04F5087051EA020317D10024E6
:104AD000012C6CDC002C09D0012C0ED1009010238D
:104AE0001A460021502001F086FF06E000901023B6
:104AF0001A460021084601F07EFF641CE8E7130017
:104B00002AD00B0028D11146012912D104F51070CA
:104B1000009010231A460021502001F06CFF04F58C
:104B20001870009010231A460021084601F063FF18
:104B300013BD022A3BD1009010231A4600210846DB
:104B400001F059FF04F52070009010231A4600214F
:104B5000502001F050FF13BD002A28D10A0026D0B2
:104B6000012A12D104F51070009010231A4600217A
:104B7000502001F040FF04F52870009010231A46E1
:104B80000021084601F037FF13BD02290FD1009024
:104B900010231A460021084601F02DFF04F530705D
:104BA000009010231A460021502001F024FF13BD6D
:104BB0007CB504460D46164612E016F8010B2E3859
:104BC000DFF8241BC0B200EB400201EB4200009072
:104BD0000523062229462046C0B201F00CFFA41D81
:104BE00030780028E9D173BDF8B504460D4600269B
:104BF0001CE00A2004E0A0F130010A29F9D2303883
:104C0000DFF8E81AC0B200EB800201EB82000090EE
:104C100010230A22002120463746FFB207EB870CFB
:104C200000EB4C00C0B201F0E6FE761C28780028AC
:104C300009D015F8010B432801D10B20E0E74528E6
:104C4000D9D10C20DCE7F1BD080000207400002061
:104C5000B0040020623400200000C8424C34002020
:104C6000643400202DE9F8438AB005460C46164608
:104C70000022142101A802F06BFE002202216846E6
:104C800003F0EAF908A80FF6A021D1E90023C0E952
:104C9000002306A80FF69821D1E90023C0E90023DC
:104CA000DFF84C8A0022284608EB80004168104655
:104CB000FFF7D3FE28460A2800F2F580DFE800F06F
:104CC000061524337A89A8B9CADCEE00DFF8240A75
:104CD00040690A2190FBF1F2C4A101A802F041F958
:104CE00001A802F057FE0746DDE0DFF8080A006978
:104CF0000A2190FBF1F2BDA101A802F032F901A84E
:104D000002F048FE0746CEE0DFF8E809C0696421FA
:104D1000B0FBF1F2B5A101A802F023F901A802F05D
:104D200039FE0746BFE000F014FD022803D000F072
:104D300010FD012807D1DFF8BC09026AABA101A868
:104D400002F00FF931E000F098FE0746BFB202F022
:104D50003DFE00EB8001B7EB410F20D300F019FEC0
:104D6000642148437F43B7FBF0F7BFB2B8F80000B7
:104D700000280DD101F033F8002809D0B8F8000060
:104D8000811CB94202DB801E874201DAA8F800705C
:104D9000B8F8002095A101A802F0E3F805E0B8F802
:104DA000002093A101A802F0DCF801A802F0F2FDB6
:104DB000074678E0DFF83C0980690A21B0FBF1F290
:104DC0008AA101A802F0CDF801A802F0E3FD074690
:104DD00069E086A7DFF81C89D8F82C000A21B0FB0F
:104DE000F1F2394601A802F0BCF8D8F82C200A20CC
:104DF000B2FBF0F000EB8001A2EB410239466846BD
:104E000002F0AFF801A802F0C5FD07467F1C4AE09A
:104E1000DFF8E008806A002805D1032277A101A805
:104E200003F05EF938E0032275A101A803F058F9F8
:104E300032E0DFF8C008406A002805D1042272A1E0
:104E400001A803F04DF915E0042270A101A803F0B8
:104E500047F90FE0DFF89C08006B002805D1042219
:104E60006BA101A803F03CF904E0042269A101A8A8
:104E700003F036F9032716E0DFF87808406B0028C6
:104E800005D1032264A101A803F02AF904E003225A
:104E900062A101A803F024F9022704E00FF69801AB
:104EA00001A802F05EF8012E5CD107F10808DFF8D6
:104EB00048687069B0F5167F48D2207801280BD178
:104EC000002257A10720FFF7C8FD002255A1404648
:104ED000C0B2FFF7C2FD1AE00FF24C1902280BD145
:104EE000002250A10720FFF7B8FD002249464046A6
:104EF000C0B2FFF7B2FD0AE0002249A10720FFF788
:104F0000ACFD002249464046C0B2FFF7A6FD052D84
:104F10000CD1002201A90820FFF79FFD012269465C
:104F2000FF1D3846C0B2FFF798FD04E0002201A93A
:104F30000820FFF792FD7069002853D14FF47A7072
:104F40007061002C4ED0002020704BE0002235A173
:104F50000720FFF782FD0022B3A14046C0B2FFF751
:104F60007CFD3FE028460A2805D1002201A9104611
:104F7000FFF773FD36E000222AA10720FFF76DFD41
:104F8000284605280BD1002201A90820FFF765FD5E
:104F900001226946F81DC0B2FFF75FFD04E0002260
:104FA00001A90820FFF759FD280001D0012D12D1D9
:104FB00008373846DFF83C17896A002905D10022F6
:104FC00008A9C0B2FFF749FD0CE0002206A9C0B253
:104FD000FFF743FD06E0002293A108373846C0B230
:104FE000FFF73BFD0BB0BDE8F08300BF2564000078
:104FF0002D2D000004070020A00A0020207B0000C7
:10500000207D0000B005002020524800204C4800C0
:105010004F464600204F4E00205600002050000012
:105020003C000000200000003E000000283400206A
:10503000B0E600082DE9F84F074600208DF8000083
:105040004FF47A74DFF8B0566C614FF47A60E86020
:1050500038460A280FD8DFE800F0068C95989B9E0A
:10506000A1A4A7AAAD00DFF88C0600F1140880699E
:10507000DFF8881688606C614FF47A60E8604FF45E
:10508000967002F090F8DFF87406394601EB4102A1
:1050900000EB8201D1F80090D1F804A0B1F808B07B
:1050A000DFF85066B16A012907D1390001D0012922
:1050B00003D1D0F87890D0F87CA001226946384618
:1050C000FFF7D0FD02F086FC002844D0D8F800207D
:1050D0001146B0F5014F02D0B0F5807F73D19245F3
:1050E00009DAA2EB0B02C8F800201046824500DB6B
:1050F0005046C8F80000D8F8000081421AD039465E
:1051000006295AD1002815D1716909B20120FFF78B
:105110000FF87061316909B20120FFF709F83061B9
:105120007069B0F57A7F00DA74613069B0F57A7F22
:1051300000DA346101208DF80000322002F033F8EB
:105140004FF47A60E8604FF4C870686101226946E4
:105150003846FFF787FD02F079FFE8680028ACD1F8
:105160004FF4FA50E860002F01D100F0EDFABDE8ED
:10517000F18FDFF8800500F110088069DFF87C15F9
:10518000486178E7DFF8788575E7DFF8788572E7BA
:10519000DFF874856FE7DFF874856CE7DFF87085FA
:1051A00069E7DFF8708566E7DFF86C8563E7DFF8AD
:1051B0006C8560E703F08AFED9E738460728B9D145
:1051C00001F0B4FCB6E7402803D048F2400398420F
:1051D000B3D14A4508DA5A44C8F800201046814540
:1051E00000DC4846C8F80000D8F80000814216D01C
:1051F000394606290ED1012811D1716909B2002062
:10520000FEF796FF7061316909B20020FEF790FF4A
:10521000306104E03846072801D101F087FC022004
:105220008DF8000089E7000020202000D80400202D
:1052300094EC0008703400202DE9F843002637462E
:105240004FF01408B14601F098FC3246114608466A
:10525000FFF708FDDFF8A05442F21070E86000F09C
:1052600084FA002802D1012000F0FAFE02F0B2FB1D
:105270000446403810D0C03806D047F64071401A76
:105280005DD0C03810D029E03046C0B2002801D02F
:10529000761E21E00A261FE03046C0B20A2801DA55
:1052A000761C19E0002617E002F0A6FB3046C0B2DB
:1052B000032807D100F04DFA04280DD000F049FA78
:1052C000052809D03046C0B2FFF7B4FE00221146CF
:1052D0003046C0B2FFF7C6FC4FF00109002C0AD0DF
:1052E00001F04BFC4FF4FA50E860002211463046C2
:1052F000C0B2FFF7B7FC02F0A9FE0A2001F053FF8D
:105300006869002805D1002211463046C0B2FFF777
:10531000A9FCA8680028A9D14FF47A70A8607F1C66
:105320004846002803D04FF0000907F1140838461A
:10533000414680B289B2884298D3BDE8F18302F039
:105340005BFB0020E860F8E744F0000860E4000838
:105350000CE5000898E5000824E60008ECE40008E5
:105360007CB504460D4650262D0110E0102106F1B3
:10537000100001F0B2FB009410231A4600213046C1
:10538000C0B201F038FB103E192001F00CFF284696
:10539000C0B28642EADA73BDF8B50C460A2093FB28
:1053A000F0F000B2642190FBF1F3DBB20E4606FB95
:1053B00013010A2291FBF2F7FFB206FB13063846EF
:1053C00000EB8001A6EB4106F6B2DFF854532878D3
:1053D000012805D10120A8600020E860287007E0BE
:1053E000022805D10020A8601020E8600020287065
:1053F0000020686026E092F8A02181F838211FE0A3
:1054000001444A4A02EB431C1CF800C081F8D8C092
:1054100002EB471C1CF800C081F8F8C002EB461CE8
:105420001CF800C081F818C10244DFF8C8C2DCF8DB
:1054300028C0BCF1010FDED192F8E02181F83821BB
:10544000401C68606868B7492246B0EB420FD7DB62
:1054500001F1D800012169600AE0009010231A468A
:1054600000212001C0B201F0C6FA6968491C6960D8
:105470006C68042CF1DDAA68E86852EA000103D0E8
:10548000002803D1102A01D10020F2BD002802D14A
:10549000521CAA6001E0401EE8600120F2BD70B518
:1054A0000546224C002104F50870FFF759FF4FF420
:1054B0007A7095FBF0F6F6B2012104EB4610FFF787
:1054C0004FFF4FF47A7000FB1655642095FBF0F601
:1054D000F6B2022104EB4610FFF742FF03216420DD
:1054E00000FB16550A2095FBF0F0C0B204EB40100B
:1054F000FFF736FF7F48806A012805D1042104F5B3
:10550000F070FFF72DFF04E0042104F5D070FFF7E1
:1055100027FF052104F51070BDE8704020E700006A
:10552000D8F10008F8F10008ECF10008C0DE00082E
:1055300010B44FF47A7392FBF3F3642492FBF4F407
:10554000A4B2002912D18018642190FBF1F14FF42C
:105550007A7290FBF2F080B29BB2984212D189B27B
:10556000A14201D0022015E0012013E0101A6421AD
:1055700090FBF1F14FF47A7290FBF2F080B29BB2A3
:10558000984201D0032005E089B2A14201D0022057
:1055900000E0012010BC70472DE9F84F0546B5F931
:1055A0000040544ED6F818805449B06A002804D1FF
:1055B000D1F80090D1F804A008E0D1F87890D1F8A3
:1055C0007CA021460020FEF7B3FD044601F0D5FA89
:1055D0002046FFF764FF484F42F21070F8606FE01A
:1055E000402803D048F24001884267D1204600B2EB
:1055F000484525DADFF828B101208BF80000224663
:1056000012B20021404680B2FFF792FF4444214687
:1056100009B2894500DA4C4623461BB2002210210C
:10562000FFF7BAFE02208BF800000021FFF746FAD0
:10563000204600B2484503D102210020FFF73EFA80
:10564000322001F0B0FD4FF47A60F86036E002F0ED
:10565000C1F9B0F5807F02D0B0F5014FC0D120462E
:1056600000B2824527DADFF8B8B001208BF80000DD
:10567000224612B20146404680B2FFF759FFA4EB22
:105680000804214609B2514500DA544623461BB2AC
:1056900000221021FFF780FE02208BF8000000217D
:1056A0000120FFF70BFA204600B2504503D101213B
:1056B0000020FFF703FA4FF47A60F86002F0C6FCAE
:1056C000F8680028C3D12146B06A012805D109B283
:1056D0000120FEF72DFD288000E02980BDE8F18F34
:1056E00030D80008C0DE0008F8F200089CED000881
:1056F000C00600207400002008000020C40800201C
:1057000090000020940000208C000020A0000020C9
:105710009C00002098000020A4000020A800002089
:10572000F4060020D80400207B2020200000000088
:105730007D20202000000000526573746F72652088
:1057400044464C54000000000020DFF8B418888460
:105750007047DFF8B00800787047DFF8A8180870C5
:105760007047DFF8A41808707047DFF89C080078CD
:1057700070472DE9FE4F0026DFF8907801223B4666
:1057800003F032FC06D834463D4606460F46CDE9C6
:10579000000104E004460D46F9E746464F46304610
:1057A000394622462B4603F01FFC33D832463B468F
:1057B0002046294603F030FC0022DFF8543803F07D
:1057C000E9FC8046894642464B4603F0E3FC8246AC
:1057D0008B46DDE9002303F0AFFDDFF83828DFF862
:1057E000383803F01BFE0BD2DFF83028DFF83038F2
:1057F00003F0FAFB04D84046494603B0BDE8F08FF9
:10580000DDE9000152465B4603F008FEC5D344467D
:105810004D46C4E70020DFF80C18EEE7DFF8E0079C
:1058200000787047DFF8D8170A784A7008700120AE
:1058300088707047DFF8F007008870473822DFF87B
:10584000EC17DFF8EC0702F03BBC38B50446FFF775
:1058500080FF022803D0FFF77CFF012873D1204688
:10586000012812D10821DFF8D00703F046FEDFF847
:10587000C4474FF48061204603F03FFE4FF480712F
:105880002046BDE8344003F038BE200012D1DFF8D6
:10589000A4474FF48071204603F02FFE0821DFF863
:1058A000980703F028FE4FF480612046BDE834409D
:1058B00003F021BE022821D1DFF87C5708212846B9
:1058C00003F01BFEDFF86C474FF48071204603F0B5
:1058D00012FE4FF48061204603F00DFE1E2001F001
:1058E00062FC0821284603F006FE1E2001F05BFC46
:1058F00008212846BDE8344003F0FFBD032C22D127
:105900000821DFF8340703F0F8FDDFF828474FF4EB
:105910008071204603F0EFFD4FF48061204603F0D4
:10592000EAFD1E2001F03FFC4FF48071204603F099
:10593000E4FD1E2001F037FC4FF480712046BDE8E5
:10594000344003F0D8BD31BD10B5032400F021F878
:10595000FFF70BFF00281BD100F08FF8B0F5167F82
:1059600002D30520FFF7F9FEFFF7F3FE002808D168
:105970002046441EC0B2002803D003F0D0FF002808
:10598000F6D100F05FFA0020BDE8104001F01FBC26
:1059900010BD2DE9F0410024254601F0F2FB06463A
:1059A00000F01DFA002803D1DFF89006006862E0DD
:1059B000204601F0E2FBDFF87C7640207861A046CB
:1059C00023E00121384603F096FD022001F0EBFBB5
:1059D000012001F0E8FB002001F0CAFB02F0E7F82B
:1059E00004190121384603F088FD022001F0DBFB99
:1059F000012001F0D8FB002001F0BAFB02F0D7F83B
:105A0000451902F023FB08F101084046C0B20A28FC
:105A1000D7DBDFF82C76DFF82486204601F0A2F9E8
:105A2000DFF8201601F0ACF90446284601F09AF997
:105A3000DFF8101601F0A4F90146204604F02AF818
:105A4000DFF8041601F024FB394601F021FB39464A
:105A500001F01EFBDFF8F41501F092F9DFF8F01504
:105A600001F08EF904F056F8C8F80000304601F055
:105A700084FBD8F80000BDE8F08138B50024254645
:105A800005E0DFF8D00504F023F904196D1C0A2D98
:105A9000F7D30A20B4FBF0F040F2BC714843000B8E
:105AA00032BDDFF85C0500218181C1810182418224
:105AB000016241610F2101830221418332218183EF
:105AC0007047F0B400210122DFF83435D881B3F9F2
:105AD0000C500646AC1B1C822F4607F11E0C844559
:105AE00005DA93F803C00CF1010C83F803C093F8B6
:105AF00003C0BCF10B0F02DB8C46C3F820C0783723
:105B0000874201DA0846D870AE4201DA0846D870FA
:105B100027463FB2B7F5967F06DA1146D8780028B7
:105B200002D1186A38181862B54207DA751B2DB20F
:105B3000332D03DB002018620146986607F11E0032
:105B40003D2800D20022B3F912507D1B1E2F02DD2A
:105B5000002D00D5002217F11E0F02DA002D00DD06
:105B600000221E8B588B4143186A414307FB0611E4
:105B7000988B454302FB051159615C82002902DCC8
:105B80000020586105E0B1F5FA6F02DD4FF4FA60CC
:105B90005861586980B2F0BC704710B402460B4699
:105BA000DFF88444884208DA9A1A192A02DB0020B6
:105BB00020800AE00220208007E0D21A192A02DCA5
:105BC0000220208001E00120208010BC7047DFF817
:105BD0003024918175E770B5064600242546C8201B
:105BE00001F0E1FA2046FFF730FEC82001F0DBFAB1
:105BF000002E2BD0DFF80804006DDFF84014096890
:105C0000484304F097F8FFF7B4FD2246DFF8483424
:105C100003F0C0FA04460D46002606E00220FFF716
:105C200014FE1E2001F0BFFA761C304680B2042814
:105C3000F4DBFFF78EFD022808D1FFF71EFF40F2CC
:105C4000A331884202D30120FFF787FDFFF781FDD2
:105C500001285AD1FFF711FF143004F06BF82246E7
:105C60002B4603F0DBFB25D2FFF707FF04F062F8B9
:105C700002460B462046294603F05EFB0022DFF871
:105C8000DC3303F0C9F904F063F880B2142190FB0F
:105C9000F1F4204680B2102800DB0F24204680B2A9
:105CA00000283CD00220FFF7D0FD1E2001F07BFA37
:105CB000641EF3E7FFF7E1FE04F03CF802460B46F2
:105CC0002046294603F0AAFB29D2FFF7D6FE14305E
:105CD00004F030F822462B4603F02EFB04F038F88F
:105CE00080B2142190FBF1F4204680B2102800DB32
:105CF0000F24204680B2002811D00320FFF7A5FD15
:105D00001E2001F050FA641EF3E71E2001F04BFA4A
:105D10000120FFF79AFD0020BDE8704095E570BDB9
:105D20001CB5C648006801F01DF8C54901F028F807
:105D30000146684603F09BFC0098002806D00199B4
:105D400089B280B2BDE81C4003F035BC03F02AFCE8
:105D5000044603F01FFC214689B280B2BDE81C4016
:105D600003F029BC10B5012802D1BDE81040D7E7E7
:105D700003F018FC044603F00DFC214689B280B202
:105D8000BDE8104003F017BC38B5FFF776FE0446B7
:105D9000A4B20A2501F01AFE6843844201D2012010
:105DA00032BDDFF8880BC06D4543A54201D2022009
:105DB00032BD002032BDDFF8781B0870002801D109
:105DC000002088607047884208D3DFF8642B506059
:105DD0009060D160002801D100201070704780B51C
:105DE000DFF84C1B087801280CD14868002809D03E
:105DF0008868B0F5FA7F03D301F0C3F9002801D019
:105E0000002002BD012002BDDFF8242B10780128FC
:105E100010D1516800290DD09068002803D09068F7
:105E20006438906070479160D06800EB8001880012
:105E300001F0A3B9704700221021DFF8F40A01F045
:105E400087BD00007CB5DFF8EC5A2E783046062876
:105E500080F2B480FFF77DFC042801D0032802D132
:105E60000720287073BDDFF8D04AE069002840F0B1
:105E7000A580761C2E70F6B2761E042E00F29E804F
:105E8000DFE806F00344657B9400FFF762FC00281E
:105E900002D00720287073BDFFF7EFFD40F25921B3
:105EA000884204D30520FFF758FC072028704FF4E0
:105EB000A060ADF8000004208DF8030003208DF8E9
:105EC00002005C4D6946284603F0C0FA0820ADF890
:105ED000000010208DF8030003208DF80200564EBC
:105EE0006946304603F0B2FA0821304603F005FB5C
:105EF0004FF48061284603F000FB4FF48071284680
:105F000003F0FBFA4FF49660E06173BD4FF4A060BC
:105F1000ADF8000010208DF8030003208DF802007A
:105F2000444D6946284603F091FA0821424803F09F
:105F3000E4FA4FF48061284603F0DFFA4FF48071F1
:105F4000284603F0DAFA4FF49670E06173BDFFF76C
:105F500094FD40F2592188421CD2FFF7FAFB002839
:105F600002D00720287073BD0220FFF7F6FB002047
:105F7000FFF76BFCC820E06173BDFFF7EAFB022866
:105F800002D00720287073BDFFF777FD40F259213A
:105F9000884205D20520FFF7E0FB0720287073BD7B
:105FA0000120FFF752FCC820E06173BDFFF765FDDB
:105FB00040F25921884201D30720287073BD38B5BB
:105FC000DFF8744940F214502062FFF7C2FB042846
:105FD00002D14FF4C870206202F038F801F0F6FCEC
:105FE0000546FFF74AFD05EB85014900814204D3D0
:105FF000206A0028F0D1012032BD002032BD00000F
:10600000440000206C3400206D3400200000F03F7C
:106010000000E03FFDA9F1D24D62503FFCA9F1D252
:106020004D6250BF0000F0BF60340020E8F300086C
:106030007400002000080140000C01404C34002096
:106040000000C8420000204100404E450000B64814
:10605000000034420028014000002440000034C009
:1060600038B504460225FFF774FB002828D0FFF757
:1060700070FB052824D0012C02D0022C21D031BD88
:106080002846C0B2002800D06D1EFFF762FB022830
:1060900003D0FFF75EFB012803D10120FFF79BFD32
:1060A00006E0FFF756FB042802D10120FFF75AFE55
:1060B000FFF785FF002803D02846C0B20028DFD1B3
:1060C00031BDFFF746FB042803D12846BDE8324026
:1060D00048E6FFF73EFB022803D0FFF73AFB012812
:1060E000EED10120BDE83240FFF7AFBB2DE9FF4103
:1060F00000270324FFF7A6FEDFF83058DFF83868E2
:10610000706A002804D1C820706203F0E1FEA87212
:10611000FFF784FB01280CD0032800F02681042817
:1061200000F07782052800F07B83082800F0C08308
:10613000FAE3A878002820D03846A870E86C00EB75
:106140008001480030613320A8850120A866286EB0
:10615000002802D00120FFF72EFE6878002817D112
:1061600000F00BFD00F022FD394605F13000FEF78E
:1061700057FA4FF4FA70B0600AE07069002807D14E
:10618000687A002804D1FEF70DFA4FF47A70706136
:106190003069002806D101F0CDFEB0F5FA7F01DAB2
:1061A0000120687200F0EDFF002801D1FFF7F1FB3C
:1061B00001F010FC0446A4B2002C00F0AE8030695F
:1061C000002800F0AA802046402861D0B0F5807FEA
:1061D00003D0B0F5014F5FD09FE0FFF7BAFA002877
:1061E00000F09B80FFF7D5FBDFF8500700686421C3
:1061F000B0FBF1F0801E09280ED300F0BEFC3A4639
:106200000FF248711046FEF728FC40F2DC5000F017
:10621000CAFF00F0B2FC80E0B84601E008F10108D6
:10622000404680B2042812DC01F0E4FC00B240F6E3
:10623000A171884200DB7F1C3846C0B20428EDDD26
:106240000320DFF8FC1608700820FFF7EBFAFFF7D1
:106250008CFA002806D1FFF77CFA052802D001202D
:10626000FFF7FEFEB5F92400002801D028850BE0D9
:10627000A86D012806D1696C09B20120FDF758FF0D
:10628000288501E0686C28850320FFF7CBFA44E0FD
:106290000520FFF7C7FA40E001F0AEFB00F06DFC0F
:1062A000DFF89886D8F80000002803D06421B0FBFE
:1062B000F1F200E03A460FF2A061684600F051FEAC
:1062C0003A4669461046FEF7C8FB684601F062FB95
:1062D0000746D8F8000000280CD06421B0FBF1F28A
:1062E00001FB1200002803D00A21B0FBF1F202E00A
:1062F000002200E0002247A1684600F032FE0122A1
:1063000069463846C0B2FEF7A8FB01F09FFE4FF485
:106310007A7000F048FF01F099FE687A002809D0F1
:1063200000F02BFC00F039FB286E002802D0002082
:10633000FFF741FDA87A002802D1002C00F0F4827A
:10634000E86C00EB8001480030613320A88500F044
:1063500009FB00F013FB00206872286E002800F093
:10636000E3820120FFF727FDDEE2A878002810D0A5
:106370003846A87000F001FC38463060E86C00EB4D
:10638000800148003061286E002802D03846FFF7AF
:1063900012FDFFF7F9FC00283ED0287901283BD0F8
:1063A000E88D401CE885384600F0E7FEFFF7D1F99C
:1063B000042807D0FFF7CDF9022803D0FFF7C9F969
:1063C00001280FD12046441EC0B200280AD0FFF792
:1063D000CCF9002802D10120FFF742FEFFF7D4FCE0
:1063E0000028EFD1FFF7D0FC012807D10520DFF806
:1063F000501508700820FFF715FA95E2FFF7C4FC66
:10640000022809D10420DFF8381508700820FFF7AA
:1064100009FA89E225640000FFF70CFA2871B5F942
:106420002810B5F9260000F06DFD122801D2288D44
:10643000E88400F0A6FE002811D101F07BFDE8847D
:10644000B5F92840B5F9267021463846FFF7A5FB77
:1064500021463846FFF7BBFB00B200F08EFE2879DC
:1064600001280BD0287A012808D100202872FFF7D4
:106470007CF9002802D10120FFF7F2FD01F0AAFA11
:106480000446A4B2204648F24001401A0ED0C0385B
:106490001BD101F0B1FA002000F06FFE00F06DFB9F
:1064A0000520FFF7BFF9002070600EE001F0A4FAAC
:1064B000002000F062FE0120FFF7B4F9FFF755F964
:1064C000002802D10220FFF7CBFD2879012802D154
:1064D0006979012902D04FF47A71B1606871B068AE
:1064E000002831D1706900282ED1A879002803D165
:1064F0000120A87100F041FBB5F92810A86D012812
:1065000013D10020FDF714FE0746B5F92610002030
:10651000FDF70EFE0A2197FBF1F109B20A2290FB6A
:10652000F2F000B2FEF7E2F80BE00A2091FBF0F186
:1065300009B2B5F926000A2290FBF2F000B2FEF78C
:10654000D5F84FF4FA707061306800282FD1B06828
:1065500000282CD0A879002803D00020A87100F0D2
:106560000CFBB5F926006885B5F928100A4602F13A
:106570001203834203DB123A904200DB6985A86D67
:10658000012805D1B5F92A100020FDF7D1FD688555
:10659000B5F92A000A2190FBF1F109B20020FDF7BC
:1065A00002FFA97A2879FEF7AFF9C8203060A87AEF
:1065B000002801D1002C04D0E86C00EB80014800D9
:1065C00030613069002816D1002000F0D6FD04208B
:1065D000FFF728F901202872288DA884FFF7C5F855
:1065E000002802D10220FFF73BFD286E002802D0D0
:1065F0000120FFF7E0FB01F00CFA012840F3948141
:1066000001F007FA042880F28F810820FFF70AF9C9
:106610008AE1A878002834D03846A8703060E86C49
:1066200000EB8001480030610120A866A86D0128B8
:1066300006D1296C09B20120FDF77AFD288501E019
:10664000286C2885286CB5F9241000290DD1696CB7
:10665000814216DAA86D012805D109B20120FDF7A3
:1066600067FD28850DE029850BE00A46824208DA9D
:10667000A86D012804D10120FDF75AFD288500E00E
:106680002985FFF7D7F8287100F07BFD00282CD171
:1066900001F050FCE884B5F92840B5F92670214690
:1066A0003846FFF77AFA287901281ED02146384665
:1066B000FFF78DFA00B200F060FD287A012814D1AE
:1066C000B5F92600B5F9281088420EDA00202872A4
:1066D000FFF74BF8002802D10120FFF7C1FC286E1C
:1066E000002802D00020FFF766FBB5F92810B5F9A5
:1066F000260000F007FC122801D2288DE8842879B2
:10670000012802D16979012902D04FF47A71B16070
:106710006871B068002834D17069002831D101F067
:1067200009FCE884A879002803D10120A87100F0B1
:1067300024FAB5F92810A86D012813D10020FDF71F
:10674000F7FC0446B5F926100020FDF7F1FC0A21FC
:1067500094FBF1F109B20A2290FBF2F000B2FDF7CE
:10676000C5FF0BE00A2091FBF0F109B2B5F9260054
:106770000A2290FBF2F000B2FDF7B8FF4FF4FA7076
:106780007061E88C68853068002821D1B0680028E5
:106790001ED0A879002803D00020A87100F0EDF9E0
:1067A000A86D012805D1B5F92A100020FDF7C0FC1D
:1067B0006885B5F92A000A2190FBF1F109B20020A1
:1067C000FDF7F1FDA97A2879FEF79EF8C820306020
:1067D00001F01FF9012803DD0820FFF723F8A3E0EB
:1067E000A87A002803D101F0F5F8002805D003208D
:1067F000FFF718F8A88C288596E03069002840F04B
:106800009380002000F0B9FC0120FFF70BF8FEF7A1
:10681000ACFF002840F088800220FFF721FC83E0D5
:106820006878012830D1286E002802D00120FFF7B7
:10683000C2FAFEF701FD434C3A464FF4A0712046E0
:1068400003F0DDF901F09CFC01F03BFF286E00280D
:1068500005D01E2141F28830FFF7B5FA03E0394632
:106860000846FFF7B0FA01224FF4A071204603F06A
:10687000C6F90120FEF7D6FFFEF777FF002853D1B7
:106880000220FFF7EDFB4FE003284DD1286E0028D2
:1068900002D00120FFF78FFA05F12800FEF77CFEF9
:1068A000288DA8842046FEF7BDFF0120A8663BE0A6
:1068B000A87800280ED03846A87000F05EF94FF492
:1068C000FA7070610120A866286E002802D0384650
:1068D000FFF771FA00F055FC002805D0384600F0AB
:1068E0004CFC40201849086001F093F8401E05D088
:1068F000401E012805D801F01DFB02E02046FEF7EE
:1069000091FF706900280FD1FDF754FF4FF4FA7022
:106910007061E879401CE871C0B2032804D13846A0
:10692000E8710120FEF77EFFBDE8FF8144000020F2
:10693000E43300206E340020080000204C34002096
:10694000B004002000280140140801402020204EFF
:106950006F2054697021000054697020523A2564F8
:106960000000000010B504463C21812003F025FC06
:106970003C212046BDE8104003F01FBC80B53C21FF
:106980008D2003F01AFC3C21142003F016FC3C215E
:10699000AF20BDE8044003F010BC80B53C218D2041
:1069A00003F00BFC3C21102003F007FC3C21AE203F
:1069B000BDE8044003F001BC10B504460A46DFF808
:1069C0008403406A002800D020343C21A2F150000A
:1069D000C0B203F0F2FB3C212046C0B2000940F0F7
:1069E000100003F0EAFB3C2104F00F042046BDE850
:1069F000104003F0E2BB2DE9F04105460C46164677
:106A00001B19DBB22046E408891000EB5171C91054
:106A1000B0EBC10000D0641C1846801003EB507826
:106A20004FEAE808069FB3EBC80302D15FFA88F883
:106A300012E008F101085FFA88F80DE02146C9B2BA
:106A40002846FFF7B9FF01233C223146384603F0C0
:106A500095FB30460744641C2046C0B24045EDDB40
:106A60003846BDE8F0812DE9F84305460F46164645
:106A7000DB19DBB23846FF08891000EB5171C910F1
:106A8000B0EBC10000D07F1C1846801003EB50799A
:106A90004FEAE909DDF82080099CB3EBC90302D174
:106AA0005FFA89F912E009F101095FFA89F90DE04D
:106AB0003946C9B22846FFF77FFF01233C22314601
:106AC000404603F05BFB204680447F1C3846C0B242
:106AD0004845EDDB4046BDE8F28378B5A1B00446F9
:106AE0000D46002201A800F033FF00260AE001A8AD
:106AF000009008232A46F100C9B22046C0B2FFF731
:106B00007AFF761C012EF2DD22B070BD80B54FF405
:106B10000040ADF8000003208DF8020010208DF831
:106B200003006946884802F091FC01BD10B5874C0E
:106B30004FF40041204602F0E0FC022000F033FB5D
:106B40004FF40041204602F0D6FC022000F02BFB5F
:106B50007F487C49496A002904D1C8214171A1219B
:106B6000417203E0C0214171A021417200233C2207
:106B70001721BDE8104003F001BB18B5A1B00022F9
:106B8000802101A800F0E4FE002409E001A80090A3
:106B900008238022E100C9B20020FFF72CFF641C0B
:106BA0002046C0B20228F1DB22B010BD2DE9F04131
:106BB000A2B001240022802102A800F0C9FE002218
:106BC0000DF1040164A001F0FDFA050000F0A880B9
:106BD0002878422840F0B28068784D2840F0AE8096
:106BE00005F136000178FF2906D14178FF2903D14C
:106BF0008078FF2800D1002400227F210DF10900B8
:106C000001F02AFA01230F2203E05B00DBB2521EDF
:106C1000D2B2082A2EDB0026374601E00C467F1C44
:106C20003846C0B20C28F0DA02EB420100EB8100DA
:106C3000284490F83EC04FF0800E4FF000082146E7
:106C40004046C0B20828E9DA704600EA0C00002984
:106C500002D1002807D001E0002804D10DF109007D
:106C6000845D1C438455761CF6B24FEA5E0E08F133
:106C70000108E5E702A800900823602200210846E9
:106C8000FFF7B9FE01F0E2F900227F210DF10900C2
:106C900001F0E2F90123002202E05B00DBB2521CAA
:106CA000082A2EDA0026374601E00C467F1C3846BB
:106CB000C0B20C28F1DAA2EB820100EB810028447B
:106CC00090F892C04FF0800E4FF0000821464046E9
:106CD000C0B20828E9DA704600EA0C00002902D1A7
:106CE000002807D001E0002804D10DF10900845DDF
:106CF0001C438455761CF6B24FEA5E0E08F101087B
:106D0000E5E702A800900823602219460020FFF75B
:106D100072FE4FF47A7000F046FA01F097F90DE038
:106D20000C4800901023602200210846FFF763FE04
:106D30004FF47A7000F037FA01F088F922B0BDE81C
:106D4000F081000074000020000C014000080140A8
:106D5000C004002084EF00084C4F474F494E2020CC
:106D6000424D500000280AD0B0FA80F18840D1F19D
:106D70009D01C905020672F1004241EB10207047E7
:106D800010B5FF2313EAD0541DBF13EAD1529C4221
:106D90009A4239E0A41ADA0780EA0103134042EA72
:106DA000012142EA0020421A3CBF641E01EB42026C
:106DB000090AB2FBF1FE01FB1E221202B2FBF1F046
:106DC00001FB10226EF30F201202B2FBF1FE4EEA1D
:106DD00000207F3406DDFE2C24DA53EA500050EB0D
:106DE000C45010BDD4F1020401FB1E2240F080719A
:106DF000192C1DDC21FA04F0C4F12004A140114338
:106E000071F10042584110BD9C421ABF03EAD152B1
:106E10009A420FE080EA010E0EF00043400004D0D9
:106E2000490016D143F0FF4010BD490008BFD343CD
:106E3000180010BD9C4205D1D21AF7D001F00041D4
:106E4000484010BD4A0212BF0846484000F00040CA
:106E500010BD4AB90902B1FA81F2914044B1A418B7
:106E6000C00140F000409EE7C90141F0004152429C
:106E70000002B0FA80F4A040141B94E7C0F3C7519D
:106E800081B1FF2906D0C110400721F0E04101F196
:106E90006051704741020CBF40F4E0016FF00041C7
:106EA0000020704700F0004100020AD0B0FA80FCD8
:106EB00000FA0CF001F16051A1EB0C5101EBD02173
:106EC000400570470CB430B583B00A4606A902915C
:106ED000044600250194009502AB01A908487844B6
:106EE0001E3003F0ADF9019A157000284EBF04461C
:106EF0000198041B204603B030BC5DF80CFB00BFBA
:106F00008B0A0000814201DA401A7047081A704764
:106F100030B40024002803D52D220A7001244042F9
:106F20000A2290FBF2F3012205E00A2593FBF5F318
:106F300002EB82056A00002BF7D1002A0CD090FBEF
:106F4000F2F303F130050D55641C02FB13031846E0
:106F50000A2392FBF3F2F0E700200855084630BC04
:106F600070470CB42DE9FC4104468846002637469C
:106F7000002C01D1304687E008AD2BE018F8060060
:106F8000E0557F1C25E0A0F57A7142F2283291424B
:106F90001FD20A2190FBF1F10A2202FB11003030CE
:106FA0002071104691FBF0F002FB10113031E170BE
:106FB0002E21A170114690FBF1F102FB110030303F
:106FC0006070104691FBF0F002FB1011303121701F
:106FD0000527761C18F80600002852D02528CDD1A8
:106FE000761C18F80600632806D0642813D066289B
:106FF0001FD0732805D0C1E755F8040BE0557F1C5E
:10700000E7E755F8041B0022885C0028E1D0E05532
:10701000521C7F1CF8E755F8040B6946FFF778FF10
:1070200000216846405C0028D3D0E055491C7F1CF5
:10703000F7E755F8040B411E0929CAD3A0F10A014C
:107040005A29C6D3A0F16401B1F5617F9BD20A2110
:1070500090FBF1F10A2202FB11003030E070104683
:1070600091FBF0F002FB10113031A1702E21617004
:10707000114690FBF1F102FB110030302070042723
:10708000A7E70020E0552046BDE8F6015DF80CFBBF
:10709000FF2212EAD05C1DBF12EAD15394459342FD
:1070A0002BE09C44D30780EA01021A4043EA002007
:1070B00043EA0121A1FB0030C04238BF40007CF10F
:1070C0007F010BDBFE294ADA5B0842EAC15153EA31
:1070D000006373F1004C51EB10207047D1F1080CA4
:1070E000DCF120012FDB5B0810FA01F10B4320FAE1
:1070F0000CF073F100415041704794451CBF02EA07
:10710000D153934280EA010202F000421DD04000B8
:1071100019D0490017D05BB9634514D00902B1FA00
:1071200081F39940BCEB030CC00140F00040C1E783
:107130000002B0FA80FC10FA0CF0B3EB0C0CC901A1
:1071400041F00041B6E71000704740000AD0490006
:1071500008D010F1807F94BF11F1807F02E042F0EF
:10716000FF407047D0437047DFF83807006B704727
:10717000DFF8341731F810007047DFF828178863FC
:107180007047DFF82007806B704700200246DFF869
:10719000143703E003EB81018A60401C0146C9B249
:1071A0000A29F7DB7047DFF8FC1600EB800290003D
:1071B0004863486B0028FCD17047DFF8E81600EB05
:1071C000800250004863486B0028FCD17047DFF80C
:1071D000DC16002808680BD120F4304040F48040D1
:1071E0000860086820F4302040F480200860704770
:1071F00020F4804040F430400860086820F480208B
:1072000040F430200860704780B503F0FDFF102087
:1072100004F084F8012004F079F8DFF8940641685E
:1072200041F4D00141F404414160016841F08071B2
:107230000160012004F001F8012004F001F8392078
:1072400004F03CF80028FAD0022003F0FCFF04F020
:1072500001F80828FBD10121052004F003F80121E1
:1072600040F20C6004F009F80121032004F010F84A
:107270000120BDE8024003F0F2BF80B501464FF0A7
:10728000006004F003F94FF4A06004F0CDF814207E
:107290008DF8000002208DF8010000208DF802001A
:1072A00001208DF80300684604F0C3F812208DF821
:1072B000000000208DF801008DF8020001208DF8FB
:1072C0000300684604F0B5F817208DF80000002090
:1072D0008DF801008DF8020001208DF8030068464A
:1072E00004F0A7F801BD38B50121DFF8C80502F0A8
:1072F00006F92020ADF8000048208DF80300DFF8E3
:10730000B8456946204602F0A1F81020ADF800000B
:1073100004208DF803006946204602F097F8052105
:10732000012002F021F91020ADF8000000208DF8B6
:107330000300DFF888556946284602F087F84FF4C5
:107340000040ADF8000003208DF8020010208DF8F9
:1073500003006946204602F079F84020ADF80000AD
:1073600003208DF8020010208DF80300694628469E
:1073700002F06CF80820ADF8000000208DF8030042
:107380006946284602F062F80420ADF800000020AB
:107390008DF803006946284602F058F80320ADF83E
:1073A000000048208DF803006946204602F04EF8A0
:1073B0000120ADF8000010208DF8030003208DF8A7
:1073C00002006946284602F041F80121284602F0F1
:1073D00094F84FF40060ADF8000003208DF802002F
:1073E00004208DF803006946284602F02FF84FF478
:1073F0008050ADF8000003208DF8020004208DF8C5
:1074000003006946284602F021F84FF40050ADF819
:10741000000003208DF8020004208DF80300694667
:10742000284602F013F84FF48040ADF80000032026
:107430008DF8020004208DF803006946284602F00A
:1074400005F84FF40070ADF8000003208DF802003D
:1074500010208DF803006946284601F0F7FF31BD82
:10746000F8B590B04FF42044DFF85454284604F0A7
:1074700021F8DFF850040590DFF82C040690002076
:107480000790022008900020099080200A904FF475
:1074900080700B904FF480600C9020200D904FF482
:1074A00000500E9000200F9005A9284604F078F8AF
:1074B0000121284604F08FF801220221284604F019
:1074C00097F8DFF80454284602F036FB00200090BD
:1074D00001208DF804008DF805004FF46027029715
:1074E0000020039002208DF810006946284602F023
:1074F00052FBDFF8D863304602F01EFB00200090FC
:1075000001208DF804008DF80500029700200390FB
:1075100001208DF810006946304602F03CFB07233D
:1075200002220421284602F094FB072301220321B2
:10753000284602F08EFB052301220221304602F08C
:1075400088FB0121284602F04FFB0121284602F06A
:1075500040FB0121304602F03CFB284602F05AFB7A
:10756000284602F05CFB002804D02046441E002878
:10757000F6D117E0304602F04DFB304602F04FFBEB
:107580000028FAD1304602F04FFB304602F051FBA2
:107590000028FAD10121284602F050FB0121304693
:1075A00002F04CFB11B0F0BDF8B54FF4E06003F011
:1075B0003BFF2F20ADF8040040F2E730ADF80800A3
:1075C0000020ADF80A00ADF8060001A94FF0804098
:1075D00004F034F801214FF0804004F08EF80122CD
:1075E00011464FF0804004F07EF801214FF08040BA
:1075F00004F06CF81C208DF8000000208DF80100CC
:1076000001208DF802008DF80300684603F011FF99
:1076100005B000BD1FB54FF4E06003F005FF2F205B
:10762000ADF804003120ADF808004FF48070ADF8DB
:107630000A000020ADF80600A54C01A9204603F081
:10764000FDFF0121204604F058F801221146204692
:1076500004F049F80121204604F038F81D208DF887
:10766000000000208DF8010001208DF802008DF847
:107670000300684603F0DDFE1FBD10B501214FF089
:10768000804004F047F80021864C08E004EB8102BA
:107690009068002802D09068401E9060491C0A291A
:1076A000F4DB8C480168491C01606078411C617002
:1076B000142803DB00F0B1F900206070A088411CA1
:1076C000A18040F2E931884203DB0020A080012044
:1076D0002070E088411CE180652815DB0020E080F7
:1076E0007D48006B00280FD0FEF73FF800280BD133
:1076F000FEF72FF8042803D0022801D0012803D177
:10770000BDE81040FEF780BB10BD70B50121704888
:1077100004F000F8634C606B002802D0606B401EE0
:1077200060636E480078002806D00020FFF720FD37
:1077300000F03DFA6A490860256C6D1C25646949B2
:10774000A06B002810D0A06B401EA063E06B401C13
:10775000E063A078002802D040224A6001E0402285
:107760000A60C043A07003E0402048600020A07081
:107770002078002812D000202070E06B00280DD067
:10778000FFF7F0FA06462846FFF7ECFA01463046C6
:10779000FFF7F6FA20630020E063206470BD10B5A7
:1077A0004A4C4FF45843594345F64D0291FBF2F1D0
:1077B0000A4692B2584345F64D0190FBF1F001465E
:1077C00089B2204602F08DFA0221204602F08CFA9E
:1077D0004549204602F07FFA01224FF4A07120466D
:1077E000BDE8104002F00BBA38B5384C4FF4A07128
:1077F000204602F08BFA00280FD0A56A204602F03E
:1078000067FA854202D30020FFF7B7FC4FF4A0715E
:107810002046BDE8344002F089BA31BD1CB5274C82
:10782000002815D00821244801F067FE4FF480613C
:10783000204601F062FE4FF48071204601F05DFEAB
:107840000121204601F059FE6420FFF7ACFC13BD76
:107850004FF48060ADF8000010208DF80300032085
:107860008DF802006946204601F0F0FD4FF480706B
:10787000ADF8000010208DF8030003208DF8020001
:107880006946204601F0E2FD4FF48071204601F088
:1078900034FE4FF48061204601F02FFE6420FFF794
:1078A00082FC13BD00000020403400200408014089
:1078B0000010024000023000000C014000080140AE
:1078C000080002404C2401400024014000280140EF
:1078D00000040040443400207400002010340020D4
:1078E000143400201008014000028000C0F3C7518A
:1078F0007E390EDDC217D1F1200106DD000240F015
:107900000040C840104450407047D04380F00040D1
:1079100070470020704730B4002513E050F8042B66
:10792000D30744BFA9F101039A18091F042942F89B
:10793000045BFAD213468C0744BF15809B1CC90711
:1079400048BF1D7050F8041B0029E7D130BC7047B8
:1079500062F30F2262F31F4200B500BF1300964688
:107960009446103928BFA0E80C50FAD85FEA417C51
:1079700028BF0CC048BF40F8042BC90728BF20F817
:10798000022B48BF00F8012B00BD0268531C0360A6
:107990001170704700F10103810704D010F8011B3A
:1079A000820781B1FAD10268A2F10131914311F04D
:1079B000803104BF50F8042FF6E709BAB1FA81F11B
:1079C00000EBD100401CC01A70470000DFF8100621
:1079D00000687047DFF80C16086800220A607047DC
:1079E000DFF8001608607047401E8041C043C00F9A
:1079F000DFF8F4150870704710B5DFF8EC4500208B
:107A00002070FFF7EDFF3220FFF7CDFB0120207043
:107A100010BDDFF8D805007870472DE9F84FDFF882
:107A2000D0050668F64306F00106DFF8BC85A8F825
:107A300004600768FF4307F00207A8F8067098F88B
:107A4000011098F80000014088F8011098F80290A1
:107A500098F8000000EA090988F80290012E07D181
:107A60000020A8F80C00B8F80800401CA8F808008E
:107A7000022F07D10020A8F80C00B8F80A00401C1B
:107A8000A8F80A00B8F80840A246BAF1190F1ADBA4
:107A900098F80000002816D0002914D0B8F80A0081
:107AA000002810D1DFF84C05406A002804D04FF4BC
:107AB0000140FFF795FF03E048F24000FFF790FF19
:107AC0000120A8F80E00B8F80A50AB46BBF1190F18
:107AD00019DB98F80000002815D0B9F1000F12D07A
:107AE000002C10D1DFF80C05406A002804D048F2C1
:107AF0004000FFF775FF03E04FF40140FFF770FF10
:107B00000120A8F81000002E26D1B8F80E00002899
:107B100017D1BAF1190F0EDA002C0CD0DFF8D4040B
:107B2000406A002804D04FF48070FFF759FF02E04C
:107B30004020FFF755FFB8F80C00401CA8F80C00D7
:107B400002E00020A8F80E00002C02D1012088F8E5
:107B500001000020A8F80800002F26D1B8F8100076
:107B6000002817D1BBF1190F0EDA002D0CD0DFF869
:107B70008404406A002803D04020FFF731FF03E06F
:107B80004FF48070FFF72CFFB8F80C00401CA8F8E9
:107B90000C0002E00020A8F81000002D02D1012006
:107BA00088F802000020A8F80A00BDE8F18F30B480
:107BB000DFF8442453681C46E4082546ADB211782A
:107BC000002905D1C000506001211170C0080FE0EC
:107BD000854201D2451B00E02D1AADB23D2D02DBDE
:107BE000C000506002E0C018001B50605068C00820
:107BF00030BC704710B50020FFF7BFFA4020DFF817
:107C0000FC1308600A20FFF7D8FADFF8F4430120DC
:107C100020700220FFF7D1FA00202070606810BDAC
:107C2000DFF8E0231178002909D1C000506001215C
:107C300011700146891000EB5170C01070475168F7
:107C400040180B469B1001EB5371A0EBE100506014
:107C50000146891000EB5170C01070472DE9F041CA
:107C600003460F464FF0640C38464008BE460021DC
:107C70001C881546AC4207D314469D1E35F8175094
:107C8000AC4201D3164609E00020BDE8F0818646EB
:107C90000A46101800EBD070401080B26246A2F184
:107CA000010C92B2002AEFD08742EDDB33F810408E
:107CB00022463546AA423DD203EB400232F8025C2E
:107CC0003246AE46724527D24FF07C57FFF74AF84E
:107CD0003946FFF7DDF9CC4903F034FD80463046E4
:107CE000FFF740F806462046FFF73CF801463046CD
:107CF00001F0D0FE3946FFF7CBF906462C1B204693
:107D000003F092FD01463046FFF73AF8014640463F
:107D1000BDE8F04101F0BEBE9542B8D1401E03F06F
:107D200083FD4FF07C51FFF7B3F9B749BDE8F0414F
:107D300003F008BD32460ED003EB40014D882946C2
:107D4000914213D33BD001467246101800EBD0701D
:107D5000401080B2A2E7FFF705F84FF07C51FFF723
:107D600097F9A949BDE8F04103F0ECBC4FF07C570E
:107D7000401C03F059FD3946FFF78AF9A24903F088
:107D8000E1FC80463046FEF7EDFF06462846FEF74A
:107D9000E9FF0146304601F07DFE3946FFF778F9EC
:107DA0000646641B204603F03FFD01463046FEF7C1
:107DB000E7FF01464046BDE8F04101F06BBE401CC4
:107DC00003F032FD4FF07C51FFF762F98E49BDE8B8
:107DD000F04103F0B7BC2DE9F041054600274FF014
:107DE0000A088A4C32E00120FFF7C2F901462068F8
:107DF0000818206022465268914200D30A46626009
:107E000022469268914200D91146A160414689B24A
:107E1000012919D16168401AA168401AC008403090
:107E2000FFF7FEFE0646280007D1324692B2A32194
:107E300004F10C00FFF712FF07460020206041F21A
:107E40008830A06000206060A8F10108404680B240
:107E50000028C8D1002D04D03046BDE8F041FEF71F
:107E600081BF3846BDE8F08170B50446684948884E
:107E70000A1D034622F81340401C488080B208289F
:107E800003DB01200870002048800878002825D0F6
:107E9000002002460D1D03E035F813301818521C5F
:107EA0001346DBB2082BF7DBFEF75CFF05464FF00D
:107EB00078563146FFF7ECF80146284601F0EAFD16
:107EC00005462046FEF74EFF294603F03BFC3146AF
:107ED000FFF7DEF8FFF70AFD80B270BD00252A46E5
:107EE00006E0081D1346DBB230F813004519521C9A
:107EF00048881346DBB20646B342F2D3FEF732FFA0
:107F000006462846FEF72EFF05463146FEF738FFA7
:107F10000146284601F0BEFD05462046FEF722FF39
:107F2000294603F00FFC3146FEF72AFFFFF7DEFC7F
:107F300080B270BD2DE9F0412C4CFDF750FF0028B8
:107F400006D1A068002803D000EB8001480044E07F
:107F5000FFF750FE05460020FFF73DFF064660682C
:107F6000281A03F061FC07462A483946FFF790F8C3
:107F70003946FFF78DF8804627483946FFF788F8DD
:107F8000414603F0DFFB254903F0DCFB314603F0FB
:107F9000D9FBFFF7ABFCA060A5F6116140F28F1290
:107FA000914203D26188491C618001E00021618017
:107FB0006188042902DD0221217001E00121217084
:107FC00040F6A1718D4201DB0321217080B2FFF7E1
:107FD0004BFFA06000EB80014800BDE8F08100008D
:107FE000BC040020483400208C0A0020B00400208B
:107FF000080C0140740000201834002014080140CF
:108000001034002020340020000080BF5C030020DA
:10801000D03300209C5349B66B9AF73DB9FC074119
:1080200010B5044645F2555003F010FC032003F050
:1080300010FC04EB84004000C00880B203F00CFC8C
:1080400003F00DFC03F010FC012010BD80B503F01F
:1080500006FC012002BD2E0062F30F2262F31F42D4
:10806000401810F0030308D0C91A1FD3DB0748BF1C
:1080700000F8012D28BF20F8022D130030B414465B
:108080001546103928BF20E93C00FAD8490728BF17
:1080900020E90C0048BF40F8042D890028BF20F8D3
:1080A000022D48BF00F8012D30BC7047C91818BF19
:1080B00000F8012DCB0728BF00F8012D7047000004
:1080C00062B38B0708D0521E11F8013B00F8013B48
:1080D00000F024808B07F6D1830740F0208000BF9A
:1080E000103A07D330B4B1E83810103AA0E838108D
:1080F000F9D230BC530724BFB1E80810A0E808103B
:1081000044BF51F8043B40F8043BD20724BF31F888
:10811000022B20F8022B44BF0B7803707047121F0C
:1081200017D35B0009D151F8043B20F8023B1B0C2C
:10813000121F20F8023BF6D20BE051F8043B00F886
:10814000013B1B0A20F8023B1B0C121F00F8013BED
:10815000F3D238BF121D521E24BF11F8013B00F8A4
:10816000013BF8D870470000002003E0491C642957
:10817000FCDB401CB0F57A7F01DA0021F7E770479D
:1081800080B54FF41852DFF8981CDFF8980CFFF711
:10819000A7FF00221021DFF8900CBDE80840FFF790
:1081A000D7BB10B4002208E0835C1C46613C1A2C4B
:1081B00001D2203B8354521C92B20B469A42F3DB0D
:1081C00010BC70472DE9FF4104460D46DFF8546CA2
:1081D00006F580674FF0000802E0203708F101083B
:1081E000404680B2102824DA0B22394601A8FFF756
:1081F00067FF0B2101A8FFF7D4FF0B22214601A83E
:1082000003F03EFB0028E8D1022207F11C012846BA
:10821000FFF756FF022207F11A016846FFF750FFE9
:10822000BDF8000006EB402000F5007004B0BDE88A
:10823000F0810020FAE70146202903D00D2901D062
:108240000A2801D1012070470020704730380A28E1
:108250008041C00F7047F8B5044600E0641C2078E8
:10826000FFF7E9FF0028F9D114F8015B2E462D2D08
:1082700001D02B2D01D114F8015B002707E007EB9B
:10828000870005EB4005303D2F4614F8015B28467A
:10829000FFF7DCFF0028F2D12D2E02D17F423846B5
:1082A000F2BD3846F2BD30B40023154604E011F8A3
:1082B000014B00F8014B5B1C1C46A4B2AC42F6D348
:1082C00030BC704770B50446FFF764FB80B20028ED
:1082D00020D02044451E00E06D1EA54204D328781E
:1082E000FFF7A9FF0028F7D100206870264600E0BC
:1082F000761C3078002803D0FFF79DFF0028F7D1C7
:10830000B44207D0AD1BAD1C2A4692B2314620467E
:10831000FFF7C9FF204670BD30B410F8013BA3F150
:1083200041041A2C00D2203311F8014BA4F141056D
:108330001A2D00D22034521E1546ADB2002D01D0A8
:10834000A342EAD01B1B06D0104680B2401E8041DB
:10835000C043C00F00E0002030BC7047F8B50646AF
:108360000F463D2106F5F07003F0BEFA002832D02A
:10837000401CFFF770FF80B2002801D001282AD1ED
:108380000446B86200250FE078610BE0A0F1D4014B
:1083900040F21D2291421ED200EB80014800002DC8
:1083A000F2D138616D1CADB2012D16DC3D2105EB1B
:1083B000850006EB001003F097FA00280BD0401C54
:1083C000FFF749FF80B2002CE0D1A0F1640140F238
:1083D0002D129142E0D30020F2BD3D2106F1A00014
:1083E00003F082FA0028F6D0401CFFF734FF80B279
:1083F000A0F13C01B1F56B7FEDD264214843F861F7
:108400003D2106F1F00003F06FFA0028E3D0401C94
:10841000FFF721FF80B2A0F110010929DBD23862F9
:108420003D2106F5A07003F05FFA0028D3D0401C70
:10843000FFF711FF80B20028CDD01A28CBDA00EB6D
:1084400080014800B8613D2106F5C87003F04CFA80
:108450000028C0D0401CFFF7FEFE80B2A0F16401EE
:108460002929B8D2F8623D2106F50C7003F03CFAD8
:108470000028B0D0401CFFF7EEFE80B2002801D0EB
:108480000128A8D178623D2106F5207003F02CFA6E
:108490000028A0D0401CFFF7DEFE80B2002801D0EB
:1084A000012898D138633D2106F5347003F01CFA99
:1084B000002890D0401CFFF7CEFE80B2002801D0EB
:1084C000012888D178630120F2BD2DE9F043ADF594
:1084D0006B7D80460D460024274622464FF44871A6
:1084E00023A8FFF735FADFF8306A4FF400724146EF
:1084F0003046FFF7E5FD1DE008F101081FFA88F896
:10850000B8F10A0F16DA06EB8800D0F80092484658
:10851000FFF740FA024692B249460EA8FFF7FCFE6A
:108520000028E9D10EA923A808EB880200EB02106D
:1085300003F0E6F9B7F5007F25DAA046224651217F
:108540000EA8FFF705FA0EA903E008F101081FFACB
:1085500088F8B8F1500FEDDAB7F5007FEADAF05D90
:1085600001F808007F1C0A2801D00D28EDD1204613
:1085700001F808000EA8FFF7A5FE9DF838000028B6
:10858000D8D0A046BCE7214601E0491C89B20A299F
:1085900007DA23A801EB81021201805C0028F4D1E4
:1085A0000124002C58D1694623A8FFF7D7FE0028E4
:1085B00000D10124002C4FD1DFF86069282204A9E2
:1085C00006F11000FFF78CFD30690A2190FBF1F2F3
:1085D0000FF6781123A8FEF7C4FC70690A2190FBFE
:1085E000F1F20FF6741137A8FEF7BBFCF0696421B5
:1085F000B0FBF1F20FF66C114BA8FEF7B2FC326A39
:108600000FF66C115FA8FEF7ACFCB0690A21B0FB55
:10861000F1F20FF6681173A8FEF7A3FCF26A0FF6E9
:10862000681187A8FEF79DFCB26A0FF668119BA837
:10863000FEF797FC726A0FF66411AFA8FEF791FC83
:10864000326B0FF66011C3A8FEF78BFC726B0FF64E
:108650006011D7A8FEF785FC00224FF4FA71284676
:10866000FFF7FAFC002C13D00026DFF8BC770A2EA7
:1086700022DA07EB8600816C284603F04DF907F1FA
:10868000140050F82610284603F046F9761CEEE751
:1086900000260FE023A806EB860100EB0111284617
:1086A00003F03AF9DFF8780850F82610284603F06E
:1086B00033F9761C0A2EEDDB20460DF56B7DBDE807
:1086C000F0832DE9F047ADF5127D0020ADF80000F4
:1086D00002464FF4FA7115A8FFF73AF9DFF83C4863
:1086E00020690A2190FBF1F20FF6600101A8FEF764
:1086F00038FC01A915A803F00FF9DFF82C576969B8
:1087000003F00AF960690A2190FBF1F20FF64801C3
:1087100001A8FEF726FC01A915A803F0FDF8A96938
:1087200003F0FAF8E0696421B0FBF1F20FF63401CE
:1087300001A8FEF716FC01A915A803F0EDF8E969F8
:1087400003F0EAF8226A0FF6280101A8FEF709FCF7
:1087500001A915A803F0E0F8296A03F0DDF8A06983
:108760000A21B0FBF1F20FF6140101A8FEF7F9FBA4
:1087700001A915A803F0D0F8696A03F0CDF8E26A00
:108780000FF6040101A8FEF7ECFB01A915A803F000
:10879000C3F8A96A03F0C0F8A26A0FF2F87101A841
:1087A000FEF7DFFB01A915A803F0B6F8E96A03F0AC
:1087B000B3F8626A0FF2E47101A8FEF7D2FB01A9D7
:1087C00015A803F0A9F8296B03F0A6F8226B0FF2A5
:1087D000D47101A8FEF7C5FB01A915A803F09CF808
:1087E000696B03F099F8626B0FF2C47101A8FEF790
:1087F000B8FB01A915A803F08FF8A96B03F08CF85A
:108800000FF2B8776A460DF102013846FFF7DAFC3D
:108810000400DFF8106622D015A8FFF7BBF8BDF8FA
:10882000001006EB411101F21C410870000A48706B
:1088300006F58060201A00F500700146491200EB31
:10884000915080120121295415A8FFF7A3F8024680
:1088500015A92046FFF734FC00F03FFA5EE00FF266
:1088600068796A460DF102014846FFF7ABFC014604
:1088700006F21644DFF8AC864FF4185A00291FD0D0
:10888000FE2215A8FFF71CFC002251463046FFF7D8
:108890005FF80C22494606F58460FFF721FCFE22B2
:1088A00015A906F50060FFF71BFC00206075C4F8F1
:1088B000208006F23A4003210170FE21817004E01D
:1088C000002251463046FFF743F80C22394606F5A0
:1088D0008060FFF705FC0FF2087706223946304624
:1088E000FFF7FEFB0622394606F50070FFF7F8FB9E
:1088F00015A8FFF74FF807463A4615A906F5C060D8
:10890000FFF7EEFB002086F80B04C4F8008002207D
:108910002071A7713F0AE77100F00CFA286C002162
:10892000C17101724171E86BC1604161C1618161D6
:1089300008460DF5127DBDE8F0872DE9F843FEB03D
:108940000020ADF800000FF274666A460DF10201D6
:108950003046FFF737FC0400DFF8C8542AD001A9DD
:10896000FFF7B3FD002800F0A48001A8FFF712F87C
:10897000BDF8001005EB411101F21C410870000A1E
:10898000487005F58060201A00F50070DFF8981433
:108990000246521200EB9250801201220A5401A8A2
:1089A000FEF7F8FF024601A92046FFF789FB00F019
:1089B00094F97EE00FF210646A460DF10201204640
:1089C000FFF700FC01004FF4185722D0FE2201A847
:1089D000FFF776FB002239462846FEF7B9FF0C2246
:1089E000214605F58460FFF77BFBFE2201A905F512
:1089F0000060FFF775FB05F2164000214175DFF8B6
:108A00002415016205F23A4003210170FE218170B4
:108A100004E0002239462846FEF79AFF0C22314630
:108A200005F58060FFF75CFB0FF2B4540622214687
:108A30002846FFF755FB0622214605F50070FFF793
:108A40004FFB0024264605F5C06921E0DFF8D80376
:108A500000EB8607D7F848804046FEF79BFF0246AA
:108A6000414609EB0400FFF72BFB4046FEF792FF5F
:108A700004197F693846FEF78DFF0246394609EB37
:108A80000400FFF71DFB3846FEF784FF0419761C2F
:108A90000A2EDBD3002085F80B0405F21640DFF820
:108AA00084140160022101718471240AC47100F0F0
:108AB00041F9DFF87403016C0022CA710A724A712D
:108AC000C06B1146C1604161C161816108467FB0E0
:108AD000BDE8F0832DE9F041ADF5027D04460E4678
:108AE0000025B6F5805F10D1DFF838534FF40072DF
:108AF000294602F0C5FE002800F0A4804FF4007261
:108B000021462846FFF7DCFA9CE0B6F5205F10D13D
:108B1000DFF814544FF40072294602F0B1FE002829
:108B200000F090804FF4007221462846FFF7C8FA03
:108B300088E0B6F5804F37D1DFF8F0634FF400726C
:108B4000314602F09DFE00287CD04FF40072214691
:108B50003046FFF7B5FAB44E012070702F4601E0A1
:108B600020347F1C3846C0B2102811DA0C2221466E
:108B70006846FFF7A5FA0B220FF24041684602F063
:108B80007FFE0028ECD1A07E7082257F012030740A
:108B9000002D06D1307C012803D1002030743080B4
:108BA00050E0012030704DE0A6F5004842F201008F
:108BB000804547D29B4FB819A0F5F4454FF4007299
:108BC0002946204602F05CFE002805D04FF40072D2
:108BD00021462846FFF774FA934C4FEA582808F1CB
:108BE0000208608A804527D105A92846FFF76DFC59
:108BF000002829D105A8FEF7CDFE618A07EB4111B7
:108C000001F577710870000A487007F58060281A2E
:108C100000F500700146491200EB915080120121CD
:108C2000215405A8FEF7B6FE024605A92846FFF71F
:108C300047FA00F052F807E0601CA6F5FC46B60AB9
:108C40000121815500F049F80DF5027DBDE8F08164
:108C500038B505460C46FFF787FA4FF40071002C33
:108C600006D10A46B2492846BDE83840FFF728BA7F
:108C7000B4F5805F06D10A466A492846BDE8384007
:108C8000FFF71EBAB4F5205F06D10A46A64928466A
:108C9000BDE83840FFF714BAB4F5804F06D10A4654
:108CA000A2492846BDE83840FFF70ABAA4F50040BB
:108CB00042F2010290420AD20A4604F1006404F52D
:108CC000064421462846BDE83840FFF7F9B900229E
:108CD0002846BDE83840FFF7BFB9F8B502F028FBD9
:108CE0000024514900E0641C102C1FD2085D0028AC
:108CF000F9D0002008554A4D15EB842002F02DFED6
:108D0000484810EB8426002700E0BF1CB7F5806FB1
:108D10000CD236F8021B17EB8420281802F00CFE48
:108D20000428F2D002F00DFB0420F2BD02F009FB92
:108D30000020F2BD38B53B4C02F0FAFA002505E000
:108D4000374800EB852002F008FE6D1C092DF7DB8B
:108D5000002501E0AD1CADB2B5F5185F09DA34F8B5
:108D6000021B2F48401902F0E7FD0428F2D004202E
:108D700032BD02F0E6FA002032BD10B52A4C236C59
:108D80001A78002A05D14002206749026167012054
:108D900018701878012833D1636CE06B8069002863
:108DA0000FD1216F1846FFF753FF40229821606CC6
:108DB00002F0E8FD4FF4E070E16B88614020A067AD
:108DC0000CE040229821A06F184402F0DBFDE06B1C
:108DD000816940398161A06F4030A0674021012046
:108DE00002F0B0FE3021012002F002FE206F403080
:108DF0002067606F403860674E4881684039816005
:108E0000606F00280AD10020E16B8861A0672067AD
:108E10000320494908700020216C087010BD000033
:108E200000000108A80A0020B000002070B5434CE3
:108E3000E36BDD694035266C3278002A06D14002AA
:108E4000E0674902C4F880100120307030780128B2
:108E500029D1002007E03A4A125C666C7254401C2B
:108E6000D969491CD961D969A942F4D3354D2888FB
:108E7000E16F4118E167D4F88020101AC4F880002F
:108E8000C00506D10020D861A1F50071606CFFF724
:108E900021FE28498A682888121A8A604FF44051B6
:108EA000022002F0BEFDD4F88000002803D0224842
:108EB0000078042808D10020E16BC861012102F08C
:108EC000C6FF0020216C087070BD000010B5FCF7D3
:108ED000B5FCFDF752FEFDF729FEFDF74EFE1A4CDC
:108EE00001202070FFF74CF9FFF7EBFB002020700A
:108EF000FFF7ACF85FF0000236A11046FBF7ADFDBE
:108F00004FF47A70FEF74FF9FFF7A0F84FF47A703C
:108F1000BDE81040FEF747B934010020740000207E
:108F2000C4000020188DDD40A80C0020A80E0020F1
:108F3000F0E80008F433002078330020B00000206F
:108F4000E43200207A3300206F34002053746254DE
:108F5000656D703D25640000576B54656D703D254F
:108F600064000000536C7054696D653D2564000019
:108F700052617465645F503D2564000054656D70F6
:108F80005374703D256400004F6666566F6C743DE7
:108F90002564000054656D703D25640048616E6471
:108FA0003D2564004C6F774375723D2564000000D9
:108FB00053686F77547970653D256400434F4E4682
:108FC00049472020545854004C4F474F494E2020C9
:108FD000424D5000436F6D706C657465642E0000E7
:108FE000F8FFFFFFFFFF00004FF4001C1CEB410FD8
:108FF00094BF1CEB430F09E041EA030C50EA4C0C10
:1090000052EA0C0C03D28B4208BF8242704714BF55
:10901000994290427047000070B44FF0004591EAC9
:10902000030F40F191816B40841A71EB030604D267
:109030006E40001BB141121973414FF4001C1CEB30
:10904000410F34BF7CEB430683E00C0DA4EB1356B9
:10905000362E00F37C80012E45EAC32341DC43EA2F
:10906000525312BFD20292025B08240545EAC12185
:1090700041EA5051D2EBC020994125D407D1B0FA32
:1090800080F610FA06F162D00020203608E0B1FA2E
:1090900081F6B140C6F1200220FA02F21143B0403D
:1090A0004FEAF474B4EB465434F001064FEA74040A
:1090B0000AD8D6F50016760D04F00044F04061FAA7
:1090C00006F25040F1404840C00A40EA415021F0C9
:1090D000004128BF5FEA500550F1000044EBD12168
:1090E00035E0DB0A45EAC121C90AB6F120050EDDEB
:1090F00042EA0242120CC5F1200603FA06F6EB40E2
:1091000042EA06056D42984161F100010DE062FA04
:1091100006F5F240554063FA06FC82EA0C02F34081
:109120005A406D42904161EB030111F4801F05D15B
:10913000641E620502D06D004041494121F4801156
:10914000430875F1004350F1000041EB045170BC3D
:1091500070471CEB410F15D223F0004352EA43063F
:109160000BD04FEA4C0CBCEB410F04D80C0D661E23
:10917000342EB7DDEBE7801A994150EA410608BF6B
:109180000021E4E708BF1CEB430F28BF6FF000018C
:10919000DDE70000B0B581EA030C0CF0004C40F2B2
:1091A000FF7515EA11541DBF15EA1357AC42AF42C3
:1091B00039E0E41923EA455343F48013C90241F02E
:1091C000004141EA505EC7021100A7FB02020028DD
:1091D0004FF00000EEFB01204FF00001E3FB072100
:1091E00018BF42F00102401800214941E3FB0E0183
:1091F000A4F580640F0302D252004041494154F16A
:1092000001046CDD470872F1004250F1000051EB9F
:109210000451A1F580115CBF41EA0C01B0BD4CEADC
:1092200005510020B0BD05EA1357AC4214BFAF4250
:1092300041E050EA410E1CBF52EA430E02E0614693
:109240000020B0BD24423C441BD15FEA070EF6D09B
:10925000090302BF01460020AEF1140EB1FA81F7F6
:10926000AEEB070401FA07FE0C37C7F1200100FA44
:1092700007F7C8404EEA000E23EA455343F4801333
:10928000A2E733F00043B3FA83F704BFB2FA82FED9
:1092900077440B3FE41BB7F1200E2FBF02FA0EF309
:1092A000BB40C7F1200E22FA0EFE38BF43EA0E0380
:1092B000BA40641C82E750EA410E14BF52EA430EE2
:1092C0006FF000014FF4001717EB430F8ABF1946E8
:1092D00017EB410FB5E74CEA05510020B0BDD4F1C2
:1092E0000104B4F120070FDAC4F12007520828BFA7
:1092F00042F0010210FA07F501FA07F7E1BF2A432D
:10930000E0403843E1400FE0352C98DCC7F1200401
:1093100052EA400220FA07F218BF42F0010231FA85
:1093200007F0A1400A43002172F1004250F1000011
:1093300051EB0C01B0BD000070B44FF0004591EA54
:10934000030F7FF571AE6B40841A71EB030603D2F5
:10935000001BB141121973414FF4001C1CEB410F6B
:1093600034BF7CEB430442E00C0DA4EB1356352EC6
:109370004FDC45EAC323DB0A45EAC121C912B6F135
:1093800020050DDD63FA05F6EB4086EA030512427F
:1093900018BF45F00105C01851F100010CD213E0CF
:1093A00062FA06F5F2405540F3415A40B340F340AB
:1093B0005A408018594107D349085FEA30005FEAF4
:1093C000350528BF45F0010501F58011420875F10A
:1093D000004250F1000041EB04514E0016F5001F11
:1093E00070BC38BF70470020090D090570471CEBA1
:1093F000410F10D252EA43060BD0BCEB410F05D807
:109400000C0DAB43661E342EB6DD02E0AB43801874
:10941000594170BC704770BC704700004FF4001C8D
:109420001CEB410F94BF1CEB430F09E041EA030C16
:1094300050EA4C0C52EA0C0C03D2994208BF9042FD
:10944000704714BF8B42824270470000F0B4002482
:10945000CA78134603F00F03D20601D58A78134366
:109460000A88D2B2002A1AD0026815E0482D12D11B
:10947000066110E00126A6400D883540B5420AD1AC
:10948000A5000F27AF40BA4303FA05F52A43CD786C
:10949000282DEBD14661641C082CEBD302600A88AE
:1094A000B2F5807F1EDB4468002218E0012602F13D
:1094B000080506FA05F50E882E40AE420ED196003C
:1094C0000F27B740BC4303FA06F63443CE78282E64
:1094D00000D14561CE78482E00D10561521C082A82
:1094E000E4D34460F0BC70470246002092680A4210
:1094F00000D001207047016170474161704770B42E
:10950000224A002801D5936900E01368C0F30344A0
:1095100085B200F44016B6F5401F06D123F0706303
:10952000146824F07064146010E0C60206D50326A7
:1095300006FA04F4A34343F0706307E00446640DA5
:10954000240105FA04F4A34343F07063002904D016
:109550000146490D09018D402B43002801D5936137
:1095600000E0136070BC704730B48A0002F00C0257
:1095700021F00301064B5C580F259540AC435C502D
:109580005C5890402043585030BC70470400014064
:1095900008000140DFF8E4048068C0F3892032212C
:1095A00048437047DFF8D4048068C0F3090000EB3B
:1095B000800148007047F8B5322290FBF2F50A208E
:1095C00091FBF0F6B6B2DFF8B444A088002801D1D0
:1095D0000220F2BD0022042104F13000FEF73CFD20
:1095E000012001E0401CC0B2A18881421ADB04EBDB
:1095F000800253681A46C2F309029B0AC3F30903A7
:109600002F46BFB2BB42EDD1236B60F31E732363C1
:10961000B2420BDB226B66F309022263226B66F314
:1096200093222263814203DA0320F2BD0420F2BDBB
:109630000320216B60F31B61216361780846E28897
:1096400060F34B22E2800120E28860F30E32E28078
:10965000E2884FF61060024042F04202E280491C6C
:1096600001F00701617000F0DFF80020F2BD2DE984
:10967000FE4F05460F46002208216846FEF768F9AE
:10968000DFF8F883B8F80400441EE4B2322601E0A3
:10969000641EE4B2002C3FD008EB8400D0F80890A0
:1096A0004846800FF4D1C9F3892A06FB0AF042F636
:1096B000E1618842ECDADFF8C803C06A64214843FC
:1096C00006FB0AF18842E3D3C9F309095046FDF7C6
:1096D00049FB0146DFF8AC03FDF7DAFC3946FDF73C
:1096E0004FFB01468B464846FDF73CFB0146DFF841
:1096F0009803FDF7CDFC594602F0F4FBC8D809EBFE
:1097000089004000019006FB0AF60096DDE90001A1
:10971000C5E90001BDE8F78FDDE90001C5E90001F9
:10972000F8E718B599B00CAA0221422000F0E7F83A
:109730000CAC6078E02801D0012073E00DF102024A
:109740000221432000F0DBF8BDF80200C0F3023133
:10975000002907D00CAA000B810001F01C01432056
:1097600000F0CDF80CA8BDF80210C1F3023100EBF7
:1097700081020421432000F0C2F80421072000F0F8
:10978000C3F8BDF80200C0F30230010011D0ADF8FB
:109790000000002007E054F820106A4602EB800227
:1097A0005160401CC0B2BDF80210C1F302318842C2
:1097B000F1DBBDF80200C0F302310A0019D100F05C
:1097C0000F02012A06D0032A08D0042A0AD0062A4A
:1097D0000CD00EE00122A94B1A700AE00222A74B1E
:1097E0001A7006E00322A54B1A7002E00422A34B74
:1097F0001A70002915D000F00F00012811D1302275
:109800006946A248FEF75CFC0420FBF7A6FFFFF7C1
:10981000C9FE0446FFF7BEFE214689B280B2FFF7BB
:10982000CAFE00201AB010BDF0B585B00022142188
:109830006846FEF78DF812208DF800006846122168
:109840004170817013218DF803108C4CE1880A4619
:10985000120B930003F01C039B1C43F08003037165
:1098600001F0EF0343710B461B0A03F001030D46A1
:109870006D0A6D0005F00E052B43120102F0700217
:109880001A43827107220023C1F3023704E0266BDA
:109890002E60121DD2B25B1C85181E46F6B2BE4267
:1098A000F5DBFF20287014206870FE20A8700F21BF
:1098B0000B2000F029F84021062000F025F8432372
:1098C0002222E088C0F3023080000A300146C9B28B
:1098D000684602F06CFC0521062000F015F807210F
:1098E0000B2000F011F805B0F0BD80B50346222230
:1098F0000121684602F026FC9DF8000002BD0346E7
:109900001046222202F01EBC80B58DF800008DF8B2
:10991000011022220221684602F0F8FB01BD38B591
:1099200000242546224630215848FEF795FB0321A6
:109930000C20FFF7E9FF3220FDF735FC03210C2056
:10994000FFF7E2FF0A20FDF72EFC0F210B20FFF7A7
:10995000DBFF641EA441E40F08D003210220FFF7BF
:10996000D3FF07210220FFF7CFFF07E003210220EA
:10997000FFF7CAFF0B210220FFF7C6FF0120FDF70A
:1099800012FC4020FFF7B1FF00F00F00022808DAB8
:109990006D1C284680B240F22D118842D9DB01208F
:1099A00032BD07210920FFF7AFFFEF210A20FFF7A3
:1099B000ABFFEF210E20FFF7A7FF01210F20FFF7DC
:1099C000A3FF002C1ED10B210220FFF79DFF2621B3
:1099D0000320FFF799FF02210C20FFF795FF0021DC
:1099E0000620FFF791FF0F210B20FFF78DFF3E2090
:1099F000FFF77BFF3F20FFF778FF4220FFF775FF5F
:109A0000002032BD07210220FFF77EFF2521032021
:109A1000FFF77AFFDFE71FB50121052001F02DFCDC
:109A200048208DF807004FF400742046ADF804007C
:109A300003208DF8060001A91548FFF707FD09214D
:109A40000020FFF791FD029401208DF80E00002008
:109A50008DF80C000C208DF80D0002A802F0CAFB56
:109A600017208DF8000001208DF801008DF802000C
:109A70008DF80300684601F0DCFC1FBD2433002094
:109A800074000020000048420000204128330020DC
:109A90000008014090EA010F41F15A8681F000412F
:109AA000421A3CBF801A89184FF0004CC0F3C752CD
:109AB000FF2A24D0C1F3C75313B3D21AD2F119032A
:109AC00027DD4CEA01214CFA03F321EA0303D140DC
:109AD000C20D4CEA0020401834BF20EA0C004CEACA
:109AE0005000D20553EA006373EB0C0C52EB1020CC
:109AF000420012F1807F38BF7047C00DC00570472B
:109B0000490212BF9A4200EB5120F8E7D2F1170345
:109B1000D9D5704700180CD2010E7F3909D4D1F184
:109B20001F015DBFC00140F00040C8406FF0000061
:109B3000704700207047000080B56E4988420BD105
:109B400001214FF4007001F0AEFB00214FF40070D2
:109B5000BDE8044001F0A7BB674988420BD1012151
:109B60004FF4806001F09FFB00214FF48060BDE85E
:109B7000044001F098BB614988420BD101214FF4A8
:109B8000004001F090FB00214FF40040BDE804408C
:109B900001F089BB01BD4368594A13400A68134369
:109BA0000A7943EA022343608368564A1340CA682D
:109BB00013438A6813434A7943EA42038360C26AC3
:109BC00022F47002097C491EC9B242EA0152C26203
:109BD00070470029816803D041F00101816070471E
:109BE00049084900816070470029816803D041F429
:109BF00080718160704721F4807181607047C9B2C3
:109C0000002A426802D011434160704722EA0101F4
:109C100041607047816841F0080181607047806849
:109C2000C00800F001007047816841F004018160C4
:109C300070478068800800F0010070470029816843
:109C400003D041F4A0018160704721F4A00181603C
:109C5000704770B407240D460A2D0BDBC568A1F1CF
:109C60000A0606EB4606B44025EA0404B340234343
:109C7000C36008E0056901EB4106B44025EA04042D
:109C8000B3402343036113461F24072B09DA436BB8
:109C9000521E02EB82029440A34391400B43436364
:109CA00014E00C2B09DC036BD21F02EB8202944000
:109CB000A34391400B43036308E0C36A0D3A02EBF0
:109CC00082029440A34391400B43C36270BC70472F
:109CD000C06C80B2704743680B4A1340194341601F
:109CE00070474162826270474268520951EA4211EC
:109CF000416070470024014000280140003C0140C1
:109D0000FFFEF0FFFDF7F1FFFFFD3FFF10B402463D
:109D1000002053680C46E4B22340126812EA112F67
:109D200002D0002B00D0012010BC7047090AC943A3
:109D300001607047014648B1B0FA80F18840C91C03
:109D4000C1F58461090501EBD02140057047000091
:109D5000C1F30A5340F2FE329B1A14DDD3F1200303
:109D60004FEAE17208DDC90241EA505141F000407A
:109D7000D84080185040704703F2E13010B1D24310
:109D800082F00040704700207047000010B56D4C15
:109D900002F0F2FA01280AD14FF4967020806A4846
:109DA00060606A48A06060688047002010BD02F0D3
:109DB00039FB012807D14FF461702080644860604E
:109DC0006448A060EFE702F0EFFB012806D15020C5
:109DD0002080614860606148A060E4E70020606026
:109DE000A060012010BDF6B583B004465C4D6F8CB9
:109DF000062638467043284403A93246FEF760F928
:109E00007F1C6F84BFB2042F04DD00206884012012
:109E100085F8200000220C216846FDF799FD69466F
:109E200095F82000002826D0002010E006FB00F264
:109E3000009BAF5EFB1800934B68AF1CBF5EFB1826
:109E40004B608B682F1DBA5ED3188B60401C0428B2
:109E5000ECDD0098052290FBF2F0ADF80C004868AC
:109E600090FBF2F0ADF80E008868114690FBF1F01F
:109E7000ADF8100025E0002011E006FB00F2009B89
:109E8000AF5EFB1800934B68AF1CBF5EFB184B60C6
:109E90008B682F1DBA5ED3188B60401C80B26A8C11
:109EA0009042EADB009890FBF2F0ADF80C004868B5
:109EB00090FBF2F0ADF80E00886890FBF2F0ADF880
:109EC0001000204603A93246FEF7FAF805B0F0BDAF
:109ED00038B584B000241B4DA96800292FD06846EE
:109EE0008847DDE900010A46014602A8FFF77BFF2B
:109EF0002888BDF90010BDF90820131A994202DB29
:109F000082188A4200DA0124BDF90210BDF90A2044
:109F1000131A994202DB82188A4201DA44F00204E1
:109F2000BDF90410BDF90C20131A994202DB801808
:109F3000884201DA44F00404204605B030BD2046D2
:109F4000FBE70000043400203DC300088FC3000875
:109F5000E9C3000839C40008CFC500080BC50008D4
:109F6000AC330020002800E0401EFDD1704780B5D2
:109F7000FCF7CCFDC020ADF8000003208DF80200F6
:109F80001C208DF8030069467B48FFF75FFA01BD8E
:109F900038B504460D462846012803D121467648A7
:109FA000FFF7A9FA002D05D121467348BDE83440DA
:109FB000FFF7A3BA31BD80B50121082001F05DF99A
:109FC000C020ADF8000014208DF8030003208DF8A8
:109FD000020069466848FFF739FA00214020FFF780
:109FE000D7FF01218020FFF7D3FF01214020FFF799
:109FF000CFFF0220FFF7B6FF00218020FFF7C8FF48
:10A000000220FFF7AFFF00214020FFF7C1FF01BD95
:10A0100080B500214020FFF7BBFF00218020FFF723
:10A02000B7FF0220FFF79EFF01214020FFF7B0FF9E
:10A030000220FFF797FF01218020FFF7A9FF0220F0
:10A04000FFF790FF00214020FFF7A2FF0220BDE8AC
:10A05000024087E738B50446082519E00021802032
:10A06000FFF796FF09E000214020FFF791FF20064F
:10A07000F4D501218020FFF78BFF0220FFF772FF4C
:10A0800001214020FFF784FF0220FFF76BFF6400EF
:10A090002846451EC0B20028E5D100214020FFF728
:10A0A00077FF01218020FFF773FFFF2400E0641E8B
:10A0B0002046C0B2002818D00220FFF753FF8021AD
:10A0C0002D48FFF711FA0028F1D101214020FFF7B8
:10A0D0005FFF0220FFF746FF00214020FFF758FFF7
:10A0E0000220FFF73FFF012032BD002032BD70B5D6
:10A0F00004460825002601218020FFF749FF16E0CD
:10A1000000214020FFF744FF0220FFF72BFF012131
:10A110004020FFF73DFF0220FFF724FF760080215B
:10A120001548FFF7E1F9002801D046F0010628465E
:10A13000451EC0B20028E3D100214020FFF728FFD0
:10A14000002C04D101218020FFF722FF03E0002131
:10A150008020FFF71DFF0220FFF704FF01214020B0
:10A16000FFF716FF0220FFF7FDFE00214020FFF75A
:10A170000FFF3046C0B270BD000C0140F8B5044678
:10A180000D4616460027002B00D04027FFF713FF8F
:10A1900076003046C0B2FFF75DFF3846FFF75AFF42
:10A1A00003E014F8010BFFF755FF2846451EC0B227
:10A1B0000028F6D1BDE8F1402AE738B504460D463F
:10A1C000FFF7F9FE6D002846C0B2FFF743FF0020FD
:10A1D000FFF740FF2046FFF73DFFBDE8314017E79E
:10A1E000F8B504460D4616461F46FFF7E4FE760016
:10A1F0003046C0B2FFF72EFF3846FFF72BFFFFF7C0
:10A20000DAFE46F001063046C0B2FFF723FF04E055
:10A210000120FFF76CFF04F8010B2846451EC0B271
:10A22000002809D02846C0B20028F1D10020FFF74D
:10A230005EFF04F8010BF0E7BDE8F140E8E600003E
:10A240002DE9F14FB0B0924604910DF142013A9AD6
:10A250002B9199464A7000200AE01AF8011B0498D5
:10A26000309A90470028049000F0B6860D98401C64
:10A270000D909AF8000050B12528EED1002100225F
:10A280000791089209910A920B910C9204E00D98A3
:10A2900000F0A4BE41F001011AF8010F2028F9D006
:10A2A00023280CD02B2804D02D2805D0302809D005
:10A2B0000BE041F00201EFE741F00401ECE741F06F
:10A2C0000801E9E741F01001E6E72A280FD1D9F8A3
:10A2D000002052F8040BC9F8002000280F9003D585
:10A2E00040420F9041F004010AF1010A14E00F927C
:10A2F000DFF828380AE00F98984205DA00EB80046E
:10A3000002EB4402303A0F920AF1010A9AF8002057
:10A31000A2F130000A28EED39AF800002E2803D0CC
:10A320004FF0FF320E9229E01AF8010F2A2809D1C6
:10A33000D9F8000050F8042BC9F800000E920AF179
:10A34000010A1BE02D280CBF0AF1010A002000229F
:10A350000E92DFF8C8470BE040B90E9AA24205DA28
:10A3600002EB820503EB4503303B0E930AF1010A31
:10A370009AF80030A3F130020A2AEDD3ADF840106C
:10A38000DFF89C07784400F5F3609AF8001001F0BC
:10A39000ABFA08B11AF8010B8DF842009DF84200A3
:10A3A000682805D19AF8000068280CD1622106E0DF
:10A3B0006C2804BF9AF800006C2804D171218DF834
:10A3C00042100AF1010A12A806901AF801BBBBF16B
:10A3D00025012CD01C3900F0D081091F022940F240
:10A3E000CC81133900F02385093900F0C681891E1C
:10A3F00000F0B885491E00F06585491E022940F22B
:10A40000BC81091F00F05E85491F00F02881491EAC
:10A4100000F00D85491E00F0D080C91E0DD0891EA8
:10A4200000F00585C91E00F0028500F0A6BD2523B9
:10A430008DF84830012100F0ABBDD9F8000050F88C
:10A44000044BC9F80000002C059440F0A3802B9920
:10A450004878002800F099804FF0FF340FF68430E0
:10A4600002F0CCF8201A40F0B78500F092BD6D1EC6
:10A4700040F0A9853096079D12AF75B1309E17F850
:10A48000012B02A9304600F073FE002801D46D1E96
:10A49000F5D10028309640F09F850A9D3020002D90
:10A4A0008DF804000CDD309E012301AA02A930467C
:10A4B00000F06EFE002840F08F856D1EF4D13096BE
:10A4C000059F089D75B1309E17F8012B02A93046F3
:10A4D00000F04EFE002801D46D1EF5D10028309604
:10A4E00040F07A850B9D3020002D8DF804000CDDA6
:10A4F000309E012301AA02A9304600F049FE00283F
:10A5000040F06A856D1EF4D1309605980899099D32
:10A51000471875B1309E17F8012B02A9304600F09C
:10A5200027FE002801D46D1EF5D10028309640F09A
:10A5300053850C9D3020002D8DF804000CDD309EDD
:10A54000012301AA02A9304600F022FE002840F0B3
:10A5500043856D1EF4D130969DF8400041077FF58C
:10A5600088AE2020002C8DF804007FF782AE309D4D
:10A57000012301AA02A9284600F00AFE002840F0A3
:10A580002B85641EF4D1309573E60FF66440059078
:10A5900000F0FFBC0E9D002D04D52046FDF7FAF912
:10A5A000044607E02A46204602F048F8002814BF77
:10A5B000041B2C46089400F0ECBCD9F8001051F8AC
:10A5C000040BC9F8001020F00004002121F0FF3531
:10A5D00012ABCDE902450593DDE9022306993C243F
:10A5E00013B90AB90E9898B102F00F053035641E00
:10A5F000EEB23A2EA8BF2735120942EA03721B09B0
:10A600000D5508BF002A03D005980D19A842EBD3B9
:10A6100008190590C4F13C020E98089282420ADAA9
:10A62000BDF84010821A4FF6EF7001400A92ADF863
:10A63000401000F0AEBC002840F1AB849DF8400013
:10A6400000F01400102840F0A4840F9B07990A988A
:10A650005B1A1B1A9A1A002A40F39B84E5E32B9994
:10A66000487820B14FF0FF340FF65430F8E69DF8EB
:10A670004200622861D0682817D06A283FD06C2831
:10A6800006D0712847D074282CD07A281DD064E0D9
:10A69000D9F8001051F8040BC9F80010002868D14F
:10A6A0004FF0FF340FF63030DAE6D9F8001051F8E9
:10A6B000040BC9F8001020B94FF0FF340FF6183022
:10A6C000CEE60D99018000F064BCD9F8001051F875
:10A6D000040BC9F8001000284BD14FF0FF340FF6DF
:10A6E000F820BDE6D9F8001051F8040BC9F80010A5
:10A6F00000283ED14FF0FF340FF6DC20B0E6D9F849
:10A70000001051F8040BC9F8001080B94FF0FF3465
:10A710000FF6C420A4E6D9F8001051F8040BC9F8CC
:10A72000001020B94FF0FF340FF6AC2098E60D9AD8
:10A73000D317C0E9002300F02CBCD9F8001051F861
:10A74000040BC9F8001020B94FF0FF340FF6882031
:10A7500086E60D99017000F01CBCD9F8001051F884
:10A76000040BC9F8001020B94FF0FF340FF6682031
:10A7700076E60D99016000F00CBCD9F80020D21DDE
:10A7800022F00702C9F80020D2E900010832C9F816
:10A790000020CDE90201C80F02D007982D210AE060
:10A7A000BDF84000810702D507982B2103E0C007C0
:10A7B00005D50798202112AA1154401C0790DDE905
:10A7C0000223079912A8CDE92C2308444BF020015D
:10A7D0006129059021AC0BD00E99002902D50621E4
:10A7E0000E9105E001BF4BF02001672901220E9276
:10A7F000DDE9022359004915491C0DD11A030BD07C
:10A80000ABF1610503211A2D089102D20FF6E41174
:10A8100010E00FF6E4110DE059004915491C0DD167
:10A820001A030BD1ABF1610503211A2D089119D33D
:10A830000FF6CC110322FDF743FCAAE3DDE9020188
:10A84000CDE92E01DDE92E2323F00047B7F5801F67
:10A8500022F000060DD20022002F08BF002E009229
:10A8600003D116E00FF69411E4E76A4601F012FFF7
:10A870000FE0DFF8DC08DFF8DC1800EB1750009081
:10A88000DDE92E234FF0FF301940DFF8CC7810407F
:10A890003943CDE902014BF0200061280DD1059824
:10A8A00030210170821CBBF1610F05920CBF782131
:10A8B000582141700798801C0790DDE9020120F0C3
:10A8C000000231F0004308BF002A02D10026002513
:10A8D00068E14BF02008B8F1610F40F0B4800E98A9
:10A8E000002847BF21210191401C0190019FDDE913
:10A8F0002C017F1C00220023DDE90245FEF78EFDBE
:10A9000000998DF8842038BF85F00045091F002F7D
:10A9100000910DF1850653DD2046294600220023D3
:10A92000FEF762FB4CD24800400D00F11C0212D031
:10A93000002A10DD40F2FF739A4206DBDFF81C1894
:10A9400005F000400143002011E06FF31E5141EA81
:10A95000025120460BE024F0000035F0004108BF12
:10A9600000280FBF29461C22294601F0CBFE0446D1
:10A970000D46FFF7EDF9FF1F002F804609DD01F0BE
:10A980005FFF02460B4620462946FEF7D5FC0446EB
:10A990000D46F01D0721B8F1000F0CDD491E5EBF0A
:10A9A00008F00F0200F8012D4FEA2818F3D502E055
:10A9B000002200F8012D491EFAD5C61D002FABDC80
:10A9C0000DF18500361A01988642D8BF304600281E
:10A9D0000DF1850430D4B04206DA0DF185010A5C30
:10A9E000082AA8BF0F2100DA0021024621AB134438
:10A9F00000E0401E13F80159521E8D42F9D00F2974
:10AA000004D10DF185018B5C5B1C8B54002A04D5AD
:10AA10000099091D21AC401C0091411E0CD4621804
:10AA2000ABF13A0613783033DDB23A2DA8BFF318F4
:10AA3000491E02F80139F5D50E99002940F1B08080
:10AA4000421E0E92ACE00099DFF8142747F29750AF
:10AA5000414391FBF2F2DDE92C45009225F00045DF
:10AA6000D2F1070204DD2046294600F04EFB0BE040
:10AA700052420020DFF8EC1600F047FB02460B467E
:10AA80002046294601F0EEFE0446B8F1660F0E9806
:10AA900006BF009F0A3706273F18142FC8BF142788
:10AAA00030200D468DF884000DF18506002F39DD2C
:10AAB0002046294601F0FAFF01460A4606F108033E
:10AAC00004200A26B2FBF6F606EB860EA2EB4E0237
:10AAD000303203F8012C0A22B6FBF2F202EB820EAE
:10AAE000A6EB4E063036401E03F8026DE9D1083F52
:10AAF000002F03F10806D9DD0846FFF71BF90246CF
:10AB00000B4620462946FEF717FC0022DFF8583690
:10AB1000FEF740FB04460D46CAE700BFCBCCCC0C89
:10AB2000544C00000DF18500361A0DF1850404E047
:10AB30000098401E761E0090641C20783028F7D0C4
:10AB4000B8F1660F02D10099491C04E0B8F1650F15
:10AB50000CBF012100210E9808188642B8BF701E54
:10AB600000281DD4B04204DA215C3429C8BF392141
:10AB700000DC30210246631E9D1800E0401E15F8DF
:10AB80000169521E8E42F9D0392902D1A15C491CBB
:10AB9000A154002A04D50099491C1C46401C009170
:10ABA0000646009D01F096FF406A0778DDF8388080
:10ABB00030B2002802DC01260FF248644BF020007E
:10ABC000662808BF6D1C16D0672846D128B210F140
:10ABD000040F48DB404546DA9DF840006D1C010734
:10ABE00003D430B24045B8BF804628B2B8EB000865
:10ABF00048BF4FF000080FFA85FBBBF1000F00F3D0
:10AC0000B5800898411C0891302205990A54B8F182
:10AC1000000F03DC9DF84000010704D50898411C93
:10AC2000089105990F5418EB0B0FB8BFC8F1000538
:10AC30002DB268420B90A84432B29045B8BF464648
:10AC4000059B089836B20996324621461844FDF70E
:10AC500037FAA8EB06000C90D2E0BBF1610F17D1D8
:10AC60004FF0700B19E030B2404504DA9DF8401007
:10AC70000A0758BF8046B8F1010848BF4FF00008E6
:10AC8000BBF1670F14BF4FF0450B4FF0650B04E0AD
:10AC9000BBF1410F08BF4FF0500B0898411C0891C1
:10ACA000B8F1000F059914F8012B0A5403DC9DF844
:10ACB000400001071AD50898411C0891B8F1000F0F
:10ACC00005990F5412DD761E30B280450598089B19
:10ACD000B8BF464632B221461844FDF7F1F908994B
:10ACE00036B271180891A8EB06000B9005980899E8
:10ACF000084429B2002980F800B003D42B22427006
:10AD0000821C04E02D2242700D46821C6D420021FF
:10AD10002CAB28460AE004460A2094FBF0F000EB36
:10AD20008005A4EB450403F8014B491C00B2002840
:10AD3000F1DC012906DC4BF02000652804BF30203F
:10AD400002F8010B00292CAB08D1302002F8010BCE
:10AD500006E0491E585C303002F8010B0029F8DC8F
:10AD6000059908980844121A099249E030B229B2AC
:10AD700088421CDA0598089B32B221461844FDF738
:10AD80009FF9089936B27118ABEB0606B8F1000FBF
:10AD900008910B9603DC9DF84000020704D5059846
:10ADA00047540999491C0991CDF8308028E005984D
:10ADB000089B2AB221461844FDF782F90898761BB1
:10ADC0005844B8F1000F089003DC9DF840100A07C2
:10ADD00003D5411C089105990F5430B28045059860
:10ADE000089BB8BF464632B204EB0B011844FDF78E
:10ADF00067F9089836B230180890A8EB06000B9057
:10AE00009DF8400000F01400102840F0C280079A1E
:10AE100008990B988A18099982180C988A18821830
:10AE20000F98824280F2B580821A0A92B1E09DF8B2
:10AE30004200622808D068280ED06A2814D06C28F6
:10AE40001FD0712810D01CE0D9F8001051F8040B65
:10AE5000C9F80010C0B21AE0D9F8001051F8040B7C
:10AE6000C9F8001080B212E0D9F80020D21D22F0FB
:10AE70000702C9F80020D2E900010832C9F8002011
:10AE800006E0D9F8001051F8040BC9F800100021B1
:10AE9000CDE902019DF8400001075AD5DDE9022302
:10AEA000002B08BF002A54D04BF02000782850D146
:10AEB000079812A930220A54401C431C079301F83A
:10AEC00000B046E09DF84200622808D068280ED005
:10AED0006A2814D06C281FD0712810D01CE0D9F833
:10AEE000001051F8040BC9F8001040B21AE0D9F86C
:10AEF000001051F8040BC9F8001000B212E0D9F8A4
:10AF00000020D21D22F00702C9F80020D2E900017A
:10AF10000832C9F8002006E0D9F8001051F8040BF7
:10AF2000C9F80010C117CDE90201002902D5079820
:10AF30002D210AE0BDF84000810702D507982B219A
:10AF400003E0C00705D50798202112AA1154401C20
:10AF5000079012A807990144059102A8594600F0EC
:10AF60004FF816E001200790D9F8000050F8041BB4
:10AF7000C9F800008DF848100BE025210122BBF133
:10AF8000000F8DF84810079203D08DF849B00221C8
:10AF900007910F9A07980A990C9C121A0898521A4E
:10AFA0000B99121A0998521A121A9DF84000141B94
:10AFB00041073FF560AA2020002C8DF804007FF7A0
:10AFC0005AAA309E2546012301AA02A9304600F064
:10AFD000DFF800283FF44BAA4FF0FF3031B0BDE856
:10AFE000F08F00007072696E74665F733A20626160
:10AFF0006420257320617267756D656E74000000B2
:10B000002DE9FC4307466F293E6908BF082405D097
:10B0100041F02000782814BF0A2410243C25D7E9E9
:10B020000023642918BF69299046994605D1002B51
:10B0300003D5D8F1000869EB4909B9F1000F08BF41
:10B04000B8F1000F0CD1386B50B9082C39D197F8F2
:10B050003800010735D530203B2586F83B0030E02D
:10B060008DF80010404649462246E31701F036FDB0
:10B070003032D0B26D1E3A28019504DB9DF80000F5
:10B08000A0F151018A187255404649462246E317FD
:10B0900001F024FD80465FEA010908BFB8F1000F06
:10B0A00003D0F86871198842DCD3082C09D197F8CD
:10B0B0003800010705D5705D302802D06D1E3020A4
:10B0C0007055C5F13C02BA617119F960386B824262
:10B0D00008DA821A3A624FF6EF70398F01403987E9
:10B0E000BDE8F38300280ED597F8380000F014006F
:10B0F000102808D17B6B7969386A5B1A1B1A9A1A77
:10B10000002AC8BF3A62BDE8F3832DE9D043064662
:10B110000F4614464FF00008DFF8509012E0E007A9
:10B1200007D542464B4630463946FEF733F80646C9
:10B130000F464046494642464B46FEF72BF8641000
:10B1400080468946002CEAD130463946BDE8D08396
:10B1500002FCFFFFFFFF0F800000E03F0000F07FD8
:10B16000A08601000000F03F84D7974100002440F2
:10B1700010B503460C461146A0689847A06020B160
:10B18000E06A401CE062002010BD4FF0FF3010BDAF
:10B19000F8B505460E4617461C4600205CB117F868
:10B1A000011BB068A847B06030B1F06A401CF06283
:10B1B0000020641EF3D1F2BD4FF0FF30F2BD00005D
:10B1C0007072696E74665F733A20256E20646973CD
:10B1D000616C6C6F776564007072696E74663A209A
:10B1E00062616420256E20617267756D656E740002
:10B1F000000000006E616E004E414E00696E6600F8
:10B20000494E4600300000003549086840F0010012
:10B2100008604A68334802404A600A68324802407F
:10B220000A60086820F480200860486820F4FE0066
:10B2300048604FF41F00886070472C4908607047D1
:10B240002C49086070472A490A68920850EA82002F
:10B25000086070472648006800F00C0070472649D7
:10B2600008607047254A0029116802D00843106021
:10B27000704721EA000010607047214A00291168D8
:10B2800002D008431060704721EA00001060704748
:10B290001C4A0029116802D008431060704721EA57
:10B2A000000010607047184A0029116802D0084356
:10B2B0001060704721EA00001060704701464009A5
:10B2C000074A012801D1106804E0022801D1106A60
:10B2D00000E0506A01F01F01C84000F00100704713
:10B2E000001002400000FFF8FFFFF6FE000042429F
:10B2F0000410024060004242D80042421410024052
:10B30000181002401C1002400C100240DFF8DC1044
:10B310000A6802F03802104308607047DFF8CC106A
:10B320000A6822F010020A600A6810430860704739
:10B33000DFF8BC00DFF8BC100160DFF8BC10016072
:10B340007047DFF8B800016841F080010160704784
:10B3500038B504464FF4302000F054F80146042973
:10B3600013D1DFF89850286840F0020028606C6024
:10B37000286840F0400028604FF4302000F042F888
:10B380002A6841F6FD710A402A6032BD70B5044654
:10B390000D464FF4005000F035F8014604290ED157
:10B3A000164E306840F00100306025804FF40050A8
:10B3B00000F028F8326841F6FE710A40326070BD34
:10B3C0000F490860704704200D490A68D20701D56B
:10B3D000012070470A68520701D5022070470968AA
:10B3E000C90600D50320704700000000002002407D
:10B3F0000420024023016745AB89EFCD10200240B5
:10B400000C20024010B50446FFF7DDFF02E0FFF715
:10B41000DAFF641E0146012901D1002CF7D1002C6E
:10B4200000D1052010BD00001B4908431B490860DE
:10B43000704770B403781C460122C17800291BD0E4
:10B4400016490B6803F4E063C3F5E0631B0A457813
:10B45000C3F104018D4081780F26DE4031400D4359
:10B460002D010F490D55017801F01F0082400D4854
:10B47000491140F8212007E003F01F0302FA03F30B
:10B480000948641140F8243070BC7047074A1140E5
:10B4900008430749086070470000FA050CED00E01A
:10B4A00000E400E000E100E080E100E080FFFF1F39
:10B4B00008ED00E002684FF6FE710A4002600021CC
:10B4C000016041608160C1604E49884205D14E48AB
:10B4D000016841F00F01016070474C49884205D175
:10B4E0004948016841F0F0010160704748498842CD
:10B4F00005D14548016841F47061016070474549D4
:10B50000884205D14048016841F4704101607047AC
:10B510004149884205D13C48016841F470210160ED
:10B5200070473E49884205D13748016841F47001AF
:10B53000016070473A49884205D13348016841F0BB
:10B540007061016070473749884205D1364801680B
:10B5500041F00F01016070473449884205D13248FB
:10B56000016841F0F001016070473149884205D11E
:10B570002D48016841F47061016070472D4988428F
:10B5800005D12948016841F47041016070472A499A
:10B59000884204D12448016841F470210160704759
:10B5A00003686FF30E138A6813430A6A13430A6928
:10B5B00013434A6913438A691343CA6913434A6AA6
:10B5C00013438A6A13430360CA6842600A68826050
:10B5D0004968C1607047002904D0016841F0010149
:10B5E0000160704702684FF6FE710A4002607047C2
:10B5F000002A026802D011430160704722EA01016B
:10B600000160704708000240040002401C00024034
:10B610003000024044000240580002406C000240EA
:10B620008000024008040240040402401C0402405E
:10B6300030040240440402405804024010B404881C
:10B64000DFF8D830984212D0DFF8E82090420ED0D0
:10B65000B0F1804F0BD0DFF8C820904207D0DFF860
:10B66000C420904203D0DFF8C020904204D14FF6AE
:10B670008F7214404A881443DFF8B020904208D0FB
:10B68000DFF8AC20904204D04FF6FF421440CA8845
:10B69000144304808A8882850A88028598420FD0E4
:10B6A000DFF8902090420BD0DFF88C20904207D03A
:10B6B000DFF88820904203D0DFF88420904201D147
:10B6C000097A01860121818210BC7047002904D0CB
:10B6D000018841F001010180704702884FF6FE7138
:10B6E0000A4002807047002A828902D0114381817A
:10B6F000704722EA010181817047002904D0018846
:10B7000041F080010180704702884FF67F710A4046
:10B7100002807047C943018270470000002C01403D
:10B720000004004000080040000C004000100040F1
:10B73000001400400034014000400140004401403A
:10B740000048014090EA010F7EF5AAA981F000416E
:10B75000431A4FF000423EBF5340C01AC91800BF01
:10B76000D3095FEAD05C13EB400F34BFB3EB410F5A
:10B7700040E07CEBD1530CD342EA012122D8D1EB3B
:10B78000402009D3400A28BF5FEA500140EBCC506B
:10B790007047401A15D04002B0FA80F2521C904017
:10B7A000400A4FEA3C23B3EB026384BF00EB730013
:10B7B00007E040F400001A16DB07C2F10102D04096
:10B7C00018437047182BFCDC31FA03F202FA03F33A
:10B7D000591A38BF42F00102D2EB40203CBF400072
:10B7E000ACF1010C5FEACC5CC20572F100414CEB9C
:10B7F0005020704713EB400F0FD2C94209D0ACEB79
:10B80000D153022B03DB4902172BDDDD7047914337
:10B81000401AC042D5D10020704713EB410FD0D35E
:10B820006FF0000070470000C2175040801AB0FA55
:10B8300080F10AD08840D1F19D01D20742EAC1517E
:10B84000020672F1004241EB10207047094908607E
:10B8500070470949086070470849086070474AF610
:10B86000AA200449086070474CF6CC4001490860A2
:10B8700070470000003000400430004008300040B5
:10B880000300002013F0030F09D0521E22BF13F84B
:10B89000010B11F801CBB0EB0C00F3D0704711F0A5
:10B8A000030F14D1121F22BF53F8040B51F804CB1D
:10B8B0006045F7D0121D0AD200BA9CFA8CFCB0EB9E
:10B8C0000C0038BF6FF0000088BF01207047521E87
:10B8D00022BF13F8010B11F801CBB0EB0C00F6D02E
:10B8E000521C08BF10467047C9B202788A421AB18A
:10B8F0001CBF10F8012FF9E718BF002070470000A7
:10B900005FEA000C11F8012B00F8012B12B111F8BD
:10B91000012BF9E760467047034600E05B1C1A788C
:10B92000002AFBD111F801CB83F800C013F8012BDA
:10B93000002AF7D17047000038B504460D4610487C
:10B94000FFF760FD052802D03420FFF739FD2946B6
:10B950002046BDE83440FFF719BD10B50446A005E8
:10B960000CD10748FFF74EFD052802D03420FFF721
:10B9700027FD2046BDE81040FFF7EABC10BD0000DF
:10B98000A086010010B40F4B03EB4103521C521070
:10B9900007E00178447841EA042123F8041B801C65
:10B9A000521EF6D110BC7047064B03EB4103521CEC
:10B9B000521004E053F8041B20F8021B521EF9D168
:10B9C00070470000006000404FF6F8710840DFF853
:10B9D000E4110860704710B4DFF8DC3153F8204000
:10B9E00048F68F121440214343F8201010BC7047D2
:10B9F00010B4DFF8C43153F82040A4B248F6BF7247
:10BA00001440CA0601D584F01004890601D584F0DB
:10BA1000200444F4004444F0800443F8204010BC67
:10BA2000704710B4DFF8903153F82040A4B24BF6C1
:10BA30008F721440CA0401D584F48054890401D55E
:10BA400084F4005444F4004444F0800443F820405B
:10BA500010BC7047DFF8602152F820304BF68F7130
:10BA60000B4083F4405343F4004343F0800342F817
:10BA700020307047DFF8402152F8203048F68F61BF
:10BA80000B4043F4004343F0800342F820307047FA
:10BA9000DFF8242152F8201049040AD552F820304A
:10BAA00048F68F710B4043F4404343F0800342F863
:10BAB00020307047DFF8002152F8201049060AD5DF
:10BAC00052F8203048F68F710B4043F4004343F0A6
:10BAD000C00342F820307047DFF8D820126892B2D5
:10BAE00002EBC002DFF8D40000EB42004908490035
:10BAF00001607047DFF8BC20126892B202EBC0020E
:10BB0000DFF8BC0000EB42004908490001607047C3
:10BB1000DFF8A010096889B201EBC001DFF89C00D2
:10BB200000EB4100006880B27047DFF888100968B8
:10BB300089B201EBC001DFF8880000EB410000682A
:10BB400080B27047DFF86C20126892B202EBC0023C
:10BB5000DFF8700000EB420001607047DFF854200E
:10BB6000126892B202EBC002DFF85C0000EB420008
:10BB70000A463F2A0ADB520911F01F0F00D1521E5C
:10BB800092B2920242F40042026070475208C90722
:10BB900000D5521C92B292020260704705490968B2
:10BBA00089B201EBC001084800EB41000068C0F316
:10BBB00009007047505C0040005C0040006000409D
:10BBC00008600040046000400C6000400146000A2C
:10BBD000C9B240EA01207047AC4890F82010891E95
:10BBE000032900D9704780B5DFE801F00C15020287
:10BBF000002180F820104FF440510220BDE804409D
:10BC0000FFF70FBFC17B282910D1816A406ABDE8C8
:10BC1000044001F0C2B80121002000F018F94FF4EF
:10BC200040510220BDE80440FFF7FBBE01BD38B51E
:10BC3000964CE57B0220FFF7B1FF60840246D821D5
:10BC40009348FFF7B1FE94F82000002802D00128A5
:10BC500003D016E0BDE831401FE02A2D05D1A16ACE
:10BC6000606ABDE8344001F0C7B8012000F01AF95D
:10BC70002421052001F089F800210220BDE834408C
:10BC8000E5E0022000F00EF92421052001F07DF806
:10BC900000210220BDE83440D9E010B500207B4CE3
:10BCA00003E07B49095C2154401C618C0A469042A8
:10BCB000F7D3784862684260A26882601F290DD07D
:10BCC000022000F0EFF8002020601A21052001F08A
:10BCD0005CF800210120BDE81040B8E0E17B282994
:10BCE00001D02A290FD1607CA27C120442EA0062B2
:10BCF000E07C42EA0022207D02436262A07DE27D78
:10BD000042EA0022A2622068634A90427AD16348E4
:10BD10000068627B904204D3A07B002801D01128E8
:10BD20000BDB022000F0BEF82421052001F02DF8E5
:10BD300000210120BDE8104089E000294AD00329F4
:10BD40002CD008295AD00A2958D012292AD01529CE
:10BD500054D01A292ED01B2928D01D294ED01E2997
:10BD600024D023292ED0252930D0282936D02A299D
:10BD70003AD02F293ED0552940D05A291ED08829A3
:10BD80003CD08A293AD08F2938D09E2936D0A8298C
:10BD900034D0AA2932D0AF2930D033E0BDE81040EA
:10BDA00000F0EABFBDE8104000F0B0BFBDE81040B1
:10BDB00000F0EFBFBDE8104000F0D6BFBDE8104076
:10BDC00000F0D6BFBDE8104000F0AFBFBDE81040A6
:10BDD00000F0BABFBDE8104001F057B8A16A606A30
:10BDE000BDE8104000F0D9BFA16A606ABDE810400C
:10BDF00001F002B8BDE8104001F02CB8BDE81040D9
:10BE000001F047B8022000F04DF82021052000F095
:10BE1000BCFF00210120BDE8104018E010B50C4621
:10BE200022469821FFF7AEFD21460120FFF78AFE4A
:10BE300030210120FFF7DCFD0320144981F82000A8
:10BE4000144881680C1B84600021017310BD10B57B
:10BE500002460C460F481249016002730D229821D8
:10BE6000FFF790FD0D210120FFF76CFE074805212B
:10BE700080F82010002C08D0042180F820103021F8
:10BE80000120BDE81040FFF7B3BD10BD58330020BE
:10BE9000E4320020F4330020555342435434002050
:10BEA0005553425380B5002803D002280ED006D344
:10BEB00001BD10210120BDE80440FFF799BD4FF4FA
:10BEC00080510220BDE80440FFF7ABBD10210120E6
:10BED000FFF78EFD4FF480510220BDE80440FFF7CC
:10BEE000A0BD00004FF0807C1CEB400F94BF1CEB0A
:10BEF000410F05E040EA010C1CEB0C0F01D281421E
:10BF0000704718BF884270470146481E0029FBD180
:10BF1000704780B501210420FFF7AFF97748012170
:10BF2000016101602220ADF8000010208DF80300AF
:10BF300003208DF8020069467148FDF787FA01BDBC
:10BF400010B56F48016821F0F0010160016841F00F
:10BF500030010160694C0120206020610320FFF75F
:10BF6000D3FF002020600320FFF7CEFF00202061D8
:10BF700010BD10B56248016821F0F0010160016850
:10BF800041F0300101605D4C002020612060032001
:10BF9000FFF7BAFF0120206120600320BDE81040B8
:10BFA000B2E738B500245648016821F0F00101607D
:10BFB000016841F080010160504D0120286003209C
:10BFC000FFF7A2FF012028610320FFF79DFF4D48E6
:10BFD0000068002808D0641C2046C0B2FB28F6DBAD
:10BFE000FFF7C7FF012032BD0020286132BD10B528
:10BFF000424C002020614248016821F0F0010160BC
:10C00000016841F030010160002020600320FFF74B
:10C010007BFF012020610320FFF776FF00202061D5
:10C0200010BD10B5354C002020613548016821F065
:10C03000F0010160016841F03001016001202060E1
:10C040000320FFF761FF012020610320FFF75CFF61
:10C050000020206110BD70B504462948016821F018
:10C06000F0010160016841F030010160234D0020C2
:10C07000286106460FE02046C0B2C009286064006F
:10C080000320FFF741FF012028610320FFF73CFF59
:10C0900000202861761C3046C0B20828EBDB70BD5A
:10C0A000F8B5044600251648016821F0F00101604A
:10C0B000016841F0800101602E46134F10E000201E
:10C0C00038600320FFF720FF012038606D000D4825
:10C0D0000068002800D06D1C0320FFF715FF761CB8
:10C0E0003046C0B20828EADB002C02D1FFF799FFE6
:10C0F00001E0FFF77CFF2846C0B2F2BD8401214277
:10C1000000080140040121429401214270B5044617
:10C110000D461646FFF714FF76003046C0B2FFF713
:10C120009AFFFFF73EFF05E014F8010BFFF793FFBE
:10C13000FFF737FF2846451EC0B20028F4D1BDE8FE
:10C14000704016E7F8B504460D4616461F46FFF741
:10C15000F7FE76003046C0B2FFF77DFFFFF721FF04
:10C160003846FFF778FFFFF71CFFFFF7E9FE46F0C0
:10C1700001063046C0B2FFF76EFFFFF712FF04E082
:10C180000120FFF78DFF04F8010B2846451EC0B2C1
:10C19000002809D02846C0B20028F1D10020FFF7BE
:10C1A0007FFF04F8010BF0E7BDE8F140E1E6F8B5E8
:10C1B00004460D4616461F46FFF7C2FE760030467F
:10C1C000C0B2FFF748FFFFF7ECFE3846FFF743FF2A
:10C1D000FFF7E7FE05E014F8010BFFF73CFFFFF760
:10C1E000E0FE2846451EC0B20028F4D1BDE8F1406B
:10C1F000BFE6000030B40468E443214A8179002995
:10C2000026D0134619680C401C605C6801688C439A
:10C210005C6004791419256801680D4325609C68E9
:10C2200001688C439C60DC6801688C43DC60417968
:10C230000468102907D199680C439C60D96800688C
:10C240000143D96009E0521810680443146004E007
:10C250000079121810680440146030BC7047024620
:10C260000020074B196811405B69134202D0002976
:10C2700000D00120704703490860704700000000AB
:10C28000000401401404014070B504460D461646F2
:10C29000FDF791FE2046FDF7DDFE2846FDF7DAFEAC
:10C2A0003046FDF7D7FEBDE87040FDF7B1BE38B5AA
:10C2B00004460D46FDF77FFE2046FDF7CBFE2846DF
:10C2C000FDF7C8FEFDF777FE44F001042046FDF7B8
:10C2D000C1FE0020FDF70BFF0446FDF799FE204646
:10C2E00032BDF8B504460D4616461F46FDF763FEFF
:10C2F0002046FDF7AFFE2846FDF7ACFEFDF75BFEDE
:10C3000044F001042046FDF7A5FE04E00120FDF7FE
:10C31000EEFE06F8010B3846471EC0B2002809D0D1
:10C320003846C0B20028F1D10020FDF7E0FE06F843
:10C33000010BF0E7BDE8F140FDF76ABE10B5012141
:10C340004C20FFF7B4FF1328F9D1242200214C2000
:10C35000FFF79AFF0520FAF726FF002408E000BF48
:10C360000DA001194A78015D4C20FFF78DFFA41C38
:10C37000102CF4D310BD000080B501214C20FFF734
:10C3800096FF132801D1012002BD002002BD024604
:10C39000062302214C20A4E70F00114C10021607BF
:10C3A00017101900218F281238B504460D46FDF7E5
:10C3B00002FE3220FDF74EFE2046FDF74BFE2846DA
:10C3C000FDF748FEBDE83140FDF722BE00B585B05F
:10C3D00003468DF80030192201216846FDF700FF61
:10C3E0009DF8000005B000BD80B500212120FFF7B9
:10C3F000DBFF40212220FFF7D7FF00212320FFF79A
:10C40000D3FF7F213020FFF7CFFF2A213220FFF713
:10C41000CBFF03213320FFF7C7FF37212020BDE8E2
:10C420000440C1E780B50F20FFF7D0FF332801D1CA
:10C43000012002BD002002BD2DE9FC410446272059
:10C44000FFF7C4FF000722D5282600276D4607E026
:10C450003046C0B2FFF7BAFF761C05F808007F1C13
:10C46000B8465FFA88F8B8F1050FF1DD68789DF8F5
:10C47000001041EA002121809DF80300A97841EADB
:10C48000002161806879297941EA0021A180BDE815
:10C49000F38170B504460D461646FDF78CFD32203B
:10C4A000FDF7D8FD2046FDF7D5FDFDF784FD3320CF
:10C4B000FDF7D0FD04E00120FDF719FE05F8010BA2
:10C4C0003046461EC0B2002809D03046C0B200280F
:10C4D000F1D10020FDF70BFE05F8010BF0E7BDE8F8
:10C4E0007040FDF795BD38B504460D46FDF763FD78
:10C4F0003220FDF7AFFD2046FDF7ACFD2846FDF7E5
:10C50000A9FDBDE83140FDF783BD7FB50446062295
:10C510000021684600F01EFD0622002102A800F05E
:10C5200019FD012269462920FFF7B3FF01220DF111
:10C5300001012820FFF7ADFF6D469DF800006978E6
:10C5400041EA002109B20911ADF8081001220DF1EC
:10C5500002012B20FFF79DFF01220DF103012A208C
:10C56000FFF797FF02AEA878E97841EA002109B207
:10C5700009117180012201A92D20FFF78AFF0122F4
:10C580000DF105012C20FFF784FF2879697941EA34
:10C59000002109B20911B180BDF80800208070881F
:10C5A0006080B088A0807FBD80B5012200216846F0
:10C5B00000F0D0FC012269460F20FFF76AFF9DF8CA
:10C5C0000000112801D1012002BD002002BD80B56C
:10C5D00037212020FFF787FF00212120FFF783FF6D
:10C5E00000212220FFF77FFF08212320FFF77BFF98
:10C5F00000212420BDE8044075E7000080B500B9A3
:10C6000006A005490B681BB122220021984701E0D2
:10C6100000F0AAFC222002BD5C340020636F6E7320
:10C62000747261696E742068616E646C65723A2020
:10C63000626164206D65737361676500C9B28307C9
:10C6400006D0521E22D310F8013B9942F7D11FE0C9
:10C65000083A13D302F1040241EA012141EA0141FF
:10C6600050F8043B121F21BF4B40A3F1013C2CEAC0
:10C67000030C1CF0803FF3D0C9B2001F083210F841
:10C68000013B521E28BF91EA030FF8D818BF0120C2
:10C69000401E704710B5144600F002F8226010BD2D
:10C6A000C1F30A5343B14A0012F5001F28D2A3F286
:10C6B000FE32A1EB0251704750EA410C20D001F04C
:10C6C000004C31EA0C01B1FA81F204BFB0FA80F3F8
:10C6D000D2180B3AB2F120032CBF00FA03F19140BB
:10C6E00041EA0C013EBFC2F1200C20FA0CF31943C1
:10C6F0009040524240F2FD33D21A01EB0351704791
:10C7000000227047124254D440F2FF7C1CEA1153BD
:10C710000FD0634531D09B1863453CBF01EB0251FC
:10C72000704701F0004141EA0C510020AFF3008056
:10C73000704750EA410320D001F0004C91EA0C010F
:10C740001CD0B1FA81F30B3B9A420DD9D21A994011
:10C7500051EA0C01C3F1200C20FA0CFC6144984012
:10C76000531C40F2FF7CD7E7914041EA0C01C2F133
:10C77000200C20FA0CF3194390407047B0FA80F374
:10C780001533202BE0D3202AEED3203A203B9A42C7
:10C7900009D9D21A00FA03F141EA0C010020531C16
:10C7A00040F2FF7CB8E700FA02F141EA0C010020F8
:10C7B0007047524240F2FF7C1CEA11530DD0634592
:10C7C000DBD0B2EB030C3CBFA1EB025170470CF184
:10C7D000010221EA035141F4801150EA410CCCD00E
:10C7E00001F0004C352A27DC30B481EA0C01B2F1AB
:10C7F000200309DAC2F12003044601FA03F5D04010
:10C800002843D1409C400CE0C3F12002450020FAAF
:10C8100003F418BF44F0010421FA03F091400C43E3
:10C82000002174F1004550F1000051EB0C0124424D
:10C8300030BC7FF47BAF70476146002076E7000094
:10C84000C11768B14840401AB0FA80F29040D21C3B
:10C85000C907C2F5846241EA025202EBD0214005C9
:10C8600070470000F0B540F2FF7581EA030C0CF050
:10C87000004C15EA11541DBF15EA1357AC42AF42E4
:10C88000E5E0BC41C1F31301C3F31303801A9941DE
:10C8900043F4801304D2641E40004941801859417A
:10C8A000C90241EA5051B1FBF3F603FB1611A2FB9A
:10C8B0000675D7EBC020A94102D2761E80185941D7
:10C8C000C90241EA5051B1FBF3FE03FB1E11A2FB6A
:10C8D0000E75D7EBC020A94103D2AEF1010E80182E
:10C8E0005941890241EA9051760546EA8E2EB1FB04
:10C8F000F3F603FB1611A2FB0675D7EB8020A941C6
:10C9000002D2761E80185941C90241EA50514EEABE
:10C91000060EB1FBF3F603FB1611A2FB0675D7EB6F
:10C92000C020A94102D2761E80185941C90241EAAD
:10C930005051B1FBF3F703FB1711A2FB0735D3EB03
:10C94000C020A94167F100070CBF004247F0010772
:10C9500066F3D5274FEA1E31B80814F5806412DD5E
:10C96000BD0775F1004250EB0E5051EB045111F52B
:10C97000801F5CBF41EA0C01F0BD4CF07F6141F0CB
:10C98000E0410020F0BDBD076D0840EA0E5041F4C3
:10C990008011D4F10104B4F120060ADAC4F12006B2
:10C9A0000200E04001FA06F3E1401843B2401543AB
:10C9B0000EE0342C13DCC6F1200445EA40056D0876
:10C9C00020FA06F2154321FA06F0A1400D4300219A
:10C9D00075F1004250F1000051EB0C01F0BD002058
:10C9E0005FEA0C01F0BDCFB992185B41B3FA83F74F
:10C9F00004BFB2FA82F6BF190B3FB7F120062FBF72
:10CA000002FA06F3BB40C7F1200622FA06F638BF49
:10CA10003343BA401CB1E419641E33E77F4231F05E
:10CA20000041B1FA81F404BFB0FA80F6A4190B3CBE
:10CA3000B4F120062FBF00FA06F1A140C4F1200690
:10CA400020FA06F638BF3143A0403C1B1AE7AC423F
:10CA50001ABF05EA1357AF4212E050EA41061CBF65
:10CA600052EA4306BFE750EA4107304661461CBF21
:10CA700041EA0551F0BD52EA430C08BFC143F0BD85
:10CA800000204FF4001616EB410F98BF16EB430F32
:10CA900008BF16EB410F24BFC14305E016EB430F5F
:10CAA0000CBF61464CEA0551F0BD0000400D49182D
:10CAB00040EA81200CD2490DA1F58061491C40F06B
:10CAC000004005DBD1F11F0154BFC840C0177047BB
:10CAD0000020704700487047540A0020BBBBE1B1FA
:10CAE000B2F5803F80F07E80022A1ED98C46B1FBD1
:10CAF000F2F102FB11C31B0443EA1043B3FBF2FC47
:10CB000002FB1C3380B240EA0343B3FBF2F002FBAA
:10CB1000103240EA0C4000237047022A05D98446AF
:10CB2000B0FBF2F002FB10C270474AB105D100F031
:10CB3000010249085FEA3000704700220023704775
:10CB400000F016BA0B00020000210020704790424E
:10CB500071EB030CF6D3B3F5803F2FD2F0B5B3FAE7
:10CB600083F7B1FA81F4A7F10F0E3D1B5340CEF1CC
:10CB7000200602FA0EF2F3415340B5F10F0746D8F2
:10CB80000F3C2C444140C4F12006A040F1414140FB
:10CB9000B1FBF3F603FB1611A2FB0645001BA941EE
:10CBA00002D2761E8018594180EA010221FA0EF362
:10CBB00062FA0EF200215A403046F0BD30B4B1FBAB
:10CBC000F3FC03FB1C11A2FB0C45001BA94103D283
:10CBD000ACF1010C8018594130BC02460B4660464E
:10CBE00000217047B2F1807F65D3F0B5B2FA82F7C9
:10CBF000B1FA81F4C7F10F063D1B22FA06F307F1E3
:10CC0000110EF24120355A40B5F10F07B8D9414015
:10CC1000C4F12006A040F1414140B1FBF3FC03FB0D
:10CC20001C11A2FB0C45001BA94103D2BCF1010C55
:10CC3000801859410F2F12D30F3FC90341EA5041C9
:10CC4000B1FBF3F603FB1611A2FB0645D4EBC03093
:10CC5000A94102D2761E8018594146EACC3C07B35E
:10CC60004140C7F12006B840F1414140B1FBF3F625
:10CC700003FB1611A2FB0645001BA94102D2761E3A
:10CC80008018594180EA010221FA0EF3C7F120040D
:10CC900062FA0EF20CFA07F05A402CFA04F1304313
:10CCA000F0BD80EA010221FA0EF3002162FA0EF2D1
:10CCB00060465A40F0BD8C46B1FBF2F102FB11C355
:10CCC0001B0243EA1063B3FBF2FC02FB1C331B02A2
:10CCD0004CEA002043EA1063B3FBF2FC02FB1C3376
:10CCE0001B024CEA002043EA1063B3FBF2FC02FB98
:10CCF0001C331B024CEA002043EA1063B3FBF2FC36
:10CD000002FB1C324CEA0020002370478849087C53
:10CD1000C00702D58748052105E08748C97C0A4637
:10CD2000252A00DB2421FFF779B88448002181807F
:10CD3000022181710021C1714172022181720021A1
:10CD4000C1720C21FFF76AB87D48002101800F21D4
:10CD50008170FF21C1700021818002218171002139
:10CD6000C1710821FFF75AB804217648FFF756B879
:10CD700008217548FFF752B86D48C17C0846132852
:10CD800000DB12217148FFF749B8704A90701173A7
:10CD9000704701210020FFF75AB870B504460D46D0
:10CDA0006B4E307800281FD12A462146282000F0FB
:10CDB0008DF800281FD05E48007B000607D50220B2
:10CDC000307029462046BDE87040FBF7D6BF0220F0
:10CDD000FFF768F824210520FFF7D7FF0121084657
:10CDE000BDE87040FFF733B8022804D12046BDE803
:10CDF0007040FBF7C2BF70BD10B50A46544C217895
:10CE000000291FD101462A2000F060F8002820D018
:10CE10004748007B000608D4012020704FF44051A1
:10CE20000220BDE81040FEF7FCBD0020FFF73AF8F5
:10CE300024210520FFF7A9FF00210120BDE81040B3
:10CE4000FFF705B8012904D11146BDE81040FBF7F2
:10CE5000EDBF10BD80B536498868002808D1087C30
:10CE6000400705D401210020BDE80440FEF7EFBFD4
:10CE70000220FFF717F824210520FFF786FF002185
:10CE80000120BDE80440FEF7E2BF01210020FEF7CB
:10CE9000DEBF80B526498868002803D10020FFF74F
:10CEA00001F809E0087B000603D50020FEF7FAFF31
:10CEB00002E00220FEF7F6FF20210520FFF765FFC4
:10CEC00000210120BDE80440FEF7C1BF80B5511824
:10CED00041F20103994211D32A2802D10220FEF720
:10CEE000E1FF0020FEF7DEFF21210520FFF74DFFC7
:10CEF00000210120FEF7ABFF002002BD0C4989682C
:10CF0000B1EB422F12D02A2803D10220FEF7CAFF2C
:10CF100002E00020FEF7C6FF24210520FFF735FFC1
:10CF200000210120FEF793FF002002BD012002BD79
:10CF30005833002030340020C0F40008480A002094
:10CF400038340020280A00202C0A0020340A00204F
:10CF50007833002010B5044610460A4601462046A4
:10CF6000FBF77AF8204610BD012000F003B800005E
:10CF70007047000080B5AFF30080024A110018200E
:10CF8000ABBEFBE72600020010B5DFF858480028CA
:10CF900004D1012021680882002010BDDFF8480874
:10CFA00000680068804720680A3010BD80B5DFF84F
:10CFB00034080168CA78DFF83408407890420DD30D
:10CFC000887800280AD18888002807D18A72DFF87B
:10CFD0001808006840688047002002BD022002BD9A
:10CFE00010B5DFF80048002804D10120216808822C
:10CFF000002010BDDFF8F0070068806880472068D7
:10D000000C3010BD10B5DFF8DC472068C1784079DE
:10D01000DFF8DC271268926990472268917A00292C
:10D0200014D0002812D1107900280FD19078002850
:10D030000CD1DFF8B4070068C068804720684179E8
:10D04000C1722068C1780173002010BD022010BD9C
:10D0500010B5DFF890170968002803D10220088274
:10D06000002010BDDFF88C4700202080087810F0E9
:10D070007F0F19D1487A0021820603D541F00201C1
:10D08000217000E021702178400609D541F00101AE
:10D090002170DFF85407006800698047204610BD02
:10D0A00001F0FE012170F4E700F07F02012A01D1B6
:10D0B000204610BD00F07F0002281BD14A7902F003
:10D0C0000F00DFF83417120651F8200008D500F0E1
:10D0D00030001028DDD1002040F001002070D8E79A
:10D0E00000F44050B0F5805FD3D1002040F0010043
:10D0F0002070CEE7002010BDF8B5DFF8E806016823
:10D10000087810F07F0005D1487A00F0DF004872FF
:10D110000020F2BD022859D14888002856D108794C
:10D12000002853D14879024622F08004DFF8C8561F
:10D13000000655F8240002D500F0300001E000F4AC
:10D140004050DFF8A8361B789C423FD200283DD0E3
:10D15000887A00283AD0100655F824000BD500F044
:10D16000300010282BD12046FEF7A4FC30212046A9
:10D17000FEF73EFC23E000F44050B0F5805F1ED186
:10D1800048F280064BF68F77002C0DD1DFF86C0645
:10D1900090F82C100020FEF7E1FC2868074087F487
:10D1A00040573E432E600AE02046FEF771FC55F8DA
:10D1B0002400074087F440573E4345F82460DFF8D9
:10D1C00028060068406980470020F2BD0220F2BDB9
:10D1D00038B5DFF8100604686079054625F080024E
:10D1E000DFF81436000653F8221002D501F03001A2
:10D1F00001E001F44051DFF8F4050078824207D2E3
:10D200006088002804D1002902D0A07A002801D12A
:10D21000022032BD48F28001280653F8224008D58A
:10D2200048F6BF70044084F01004214343F82210F4
:10D2300007E04BF68F70044084F48054214343F898
:10D240002210DFF8A405006880698047002032BD05
:10D2500080B5DFF890050068417A41F02001417205
:10D26000DFF884050068C0698047002002BDDFF850
:10D2700074251268538A002804D18888C31A13823F
:10D2800000207047086818447047F8B5DFF8545517
:10D29000286800F110063488B168002916D0002CE7
:10D2A00014D0B088844200D90446204688470746F7
:10D2B0003088001B30807088201870800020FEF7B6
:10D2C00034FC224601463846FEF76EFB30880028C3
:10D2D0000CD04FF44050DFF8281508800021084694
:10D2E000FEF730FC3020DFF81C1508803088B1884C
:10D2F000884203D3032029680872F1BD002803D0B7
:10D30000052029680872F1BD10D10620296808722D
:10D310000020DFF8F414096889B2DFF8F02402EB8A
:10D32000410210603020DFF8DC140880F1BD2DE9E7
:10D33000F041DFF8B054286800F110073C88002C59
:10D340001DD1007A04281AD1DFF8B804DFF8C01420
:10D350000A78012A0FD10022DFF8AC341B689BB297
:10D36000DFF8A84404EB4304226030220280042644
:10D37000002008702BE007261021018027E0B888E4
:10D38000A04201D3042600E00226844200D90446CC
:10D390002046B968884780460020FEF7B9FB224640
:10D3A00001464046FEF7EEFA21460020FEF7CAFB92
:10D3B0003888001B3880788824187C803020DFF87B
:10D3C000441408804FF44050DFF834140880286873
:10D3D0000672BDE8F08138B50220DFF80844226803
:10D3E0005578117811F07F0F2DD1092D02D1FFF75B
:10D3F000DDFD3EE0052D0FD1D0787F2808DC907848
:10D40000002805D19088002802D1907A002801D008
:10D4100008204EE000202CE0032D08D1D17801290E
:10D4200027D19188002924D1FFF712FF21E0012D97
:10D430001FD1D17801291CD19188002919D1517AA5
:10D4400089060FD415E001F07F02012A04D10B2DCB
:10D450000FD1FFF7D7FD0CE001F07F01022908D1C1
:10D46000012D02D1FFF748FE03E0032D01D1FFF7A4
:10D47000AFFE01000AD02846DFF874130968496935
:10D4800088470146032901D1092012E0002801D074
:10D4900008200EE006200021DFF86C23126892B20B
:10D4A000DFF8683303EB420319603021DFF85423BF
:10D4B00011802168087231BD38B5DFF82843226831
:10D4C0005178002506291AD1107810F07F0F40F00E
:10D4D0007F809078012804D1DFF814030068C569C3
:10D4E00076E0022804D1DFF808030068056A6FE0DF
:10D4F00003286DD1DFF8F8020068456A68E000296A
:10D5000042D1508800283FD1D08802283CD11079E0
:10D51000002839D1117811F07F0F05D190880028AB
:10D5200002D1DFF8F05253E001F07F0001280DD165
:10D5300029465079AE4A126892699047002847D12F
:10D540002068807A002843D0B24D41E001F07F018D
:10D5500002293DD15379194601F00F0201F0700103
:10D56000A5481B0650F8220002D500F0300001E06B
:10D5700000F440509D4B1B789A4229D2002927D1B4
:10D58000002825D0A34D23E0082905D1107810F0FC
:10D590007F0F1DD1A04D1BE00A2919D1107800F092
:10D5A0007F00012814D1907A002811D050880028DB
:10D5B0000ED1107900280BD1D088012808D1294636
:10D5C00050798B4A126892699047002800D1934D98
:10D5D0002068290007D00021418220688561084623
:10D5E000A847002107E04078814909680969884710
:10D5F0000146032805D02268108A4FF6FF7398422F
:10D6000003D109202168087231BD022901D0002808
:10D6100002D10820107231BD1178090629D5D188B0
:10D620000B460093009B0546AB4202D20098108245
:10D6300016E0884214D26E49096891F82C1002460F
:10D640000B469A4203D200207149087008E090FB13
:10D65000F1F201FB1200002802D101206C49087090
:10D660006348006890F82C0021688882BDE831404A
:10D670005DE6032010724FF440506149088031BDCF
:10D6800038B56148006880B2654901EB40010888FF
:10D69000644911EB4004534D2868017A092911D0DF
:10D6A00021780170607829684870A088FEF78EFAAA
:10D6B000296848802089FEF789FA29688880A0892E
:10D6C0002968C8800120296808722868C088002855
:10D6D00002D1FFF780FE01E0FFF7EEFEBDE831402A
:10D6E00048E010B53F4C2068017A022901D0042996
:10D6F00004D1FFF71CFE2068007A16E0062913D13A
:10D70000417805290AD1017811F07F0F06D1C07840
:10D7100000F04AF834480068006A804734480068DE
:10D7200080688047082000E0082021680872BDE872
:10D7300010401FE010B52B4C2068007A022801D061
:10D74000042801D1082011E0032801D0052804D1C4
:10D75000FFF79BFD2068007A08E0072805D12448E0
:10D760000068C0688047082000E00820216808722F
:10D77000BDE8104080B5214890F82C100020FEF73D
:10D78000EDF918480068017A082906D14FF4805154
:10D790001B4A118010211B4A1180007A092801D1EF
:10D7A000012002BD002002BD70B41049097800229A
:10D7B000114C48F68F760CE01346DBB254F8235038
:10D7C00035401D4345F4004545F0800544F823509D
:10D7D000521C8A42F0D340F080001349086070BCAC
:10D7E00070470000A0330020A83300209E0A0020CC
:10D7F000A433002066340020005C00409C09002017
:10D800005034002052340020505C0040046000403E
:10D810007134002051D0000889CF0008E1CF000802
:10D8200008600040006000404C5C00407047000011
:10D8300000000000000000000000000000000000E8
:10D84000000070F8F87000000000000D0D000000EE
:10D8500000383800003838000000000000000000E8
:10D860000020F8F820F8F82000020F0F020F0F0236
:10D87000003078CE8E18100000040C38390F0600E6
:10D88000183C24BCD86030000006030D1E121E0C8C
:10D8900000B0F8487830000000070F0809070F09AA
:10D8A0000000003838000000000000000000000008
:10D8B0000000C0F0380800000000071F38200000FA
:10D8C00000000838F0C00000000020381F070000EA
:10D8D0000080A0E0C0E0A08000000203010302007D
:10D8E000008080E0E0808000000000030300000072
:10D8F00000000000000000000000002C3C1C0000A4
:10D900000080808080808000000000000000000017
:10D9100000000000000000000000000C0C0C0000E3
:10D9200000000080E078180000181E0701000000C9
:10D930000000F0F80868F8F00000070F0B080F0768
:10D9400000202030F8F80000000000000F0F000059
:10D950000030380888F87000000C0E0B0908080029
:10D960000030388888F8700000060E08080F07009D
:10D970000000F8F800E0E00000030302020F0F02CD
:10D9800000F8F88888880800000808080C070300D9
:10D9900000C0E07858C8800000070F08080F070093
:10D9A00000080888E878180000000E0F0100000049
:10D9B0000070F8C888F8700000070F08090F07000A
:10D9C00000F0F80808F8F0000000090D0F0301004E
:10D9D00000000060606000000000000C0C0C000003
:10D9E00000000060606000000000002C3C1C000093
:10D9F0000080C0603018080000000103060C080019
:10DA00000040404040404000000101010101010090
:10DA10000008183060C0800000080C0603010000F8
:10DA200000303888C87830000000000D0D0000007C
:10DA3000F0F80888C848F8F0070F08090B0A0B0B24
:10DA400000E0F01818F0E000000F0F01010F0F00C8
:10DA500000F8F88888F87000000F0F08080F07001A
:10DA600000F0F8080838300000070F08080E06001C
:10DA700000F8F80818F0E000000F0F080C0703008A
:10DA800000F8F88888880800000F0F0808080800C8
:10DA900000F8F88888880800000F0F0000000000D8
:10DAA00000F0F8080838300000070F08090F0F00D1
:10DAB00000F8F88080F8F800000F0F00000F0F004A
:10DAC000000008F8F80800000000080F0F08000028
:10DAD0000000000000F8F80000060E08080F07001C
:10DAE00000F8F880E0781800000F0F00030F0C001A
:10DAF00000F8F80000000000000F0F0808080800F8
:10DB000000F8F820C020F8F8000F0F0001000F0FF8
:10DB100000F8F860C080F8F8000F0F0000010F0F48
:10DB200000F0F80808F8F00000070F08080F0700D9
:10DB300000F8F88888F87000000F0F00000000005F
:10DB400000F0F80808F8F00000070F08183F270059
:10DB500000F8F88888F87000000F0F00010F0E0021
:10DB6000003078C88818100000040C08090F06005F
:10DB7000000808F8F80808000000000F0F00000077
:10DB800000F8F80000F8F80000070F08080F070079
:10DB900000F8F80000F8F8000003070C0C07030079
:10DBA00000F8F800C000F8F800010F0E010E0F0198
:10DBB000001838E0C0381800000E0F00010F0E00EA
:10DBC0000078F88080F878000000000F0F00000057
:10DBD00000080888C8783800000E0F0908080800F7
:10DBE0000000F8F80808000000007F7F40400000B7
:10DBF000001878E08000000000000001071E1800F7
:10DC000000000808F8F80000000040407F7F000096
:10DC10003018081830203018000000000000000004
:10DC200000000000000000004040404040404040F4
:10DC3000000002060E0800000000000000000000C6
:10DC40000000202020E0C00000060F09090F0F008F
:10DC500000F8F82020E0C000000F0F08080F0700B0
:10DC600000C0E0202060400000070F08080C0400FE
:10DC700000C0E02020F8F80000070F08080F0F0090
:10DC800000C0E02020E0C00000070F0909090100E2
:10DC90000080F0F88888880000000F0F0000000066
:10DCA00000C0E02020E0E00000474F48487F3F00F0
:10DCB00000F8F82020E0C000000F0F00000F0F0058
:10DCC000002020ECEC0000000008080F0F080800FE
:10DCD00000002020ECEC0000004040407F3F0000AE
:10DCE00000F8F80080E06000000F0F01030E0C0048
:10DCF000000808F8F80000000008080F0F080800E6
:10DD000000E0E020E020E0C0000F0F0007000F0F50
:10DD100000E0E02020E0C000000F0F00000F0F0027
:10DD200000C0E02020E0C00000070F08080F070037
:10DD300000E0E02020E0C000007F7F08080F07001F
:10DD400000C0E02020E0E00000070F08087F7F000F
:10DD500000E0E08040606000000F0F000000000065
:10DD600000C0E0202020200000080909090F06005B
:10DD70000020F8F8202020000000070F0808080005
:10DD800000E0E00000E0E00000070F08080F0F00CF
:10DD900000E0E00000E0E0000003070C0C070300D7
:10DDA00000E0E000C000E0E000030F0C030C0F03F4
:10DDB0000060E08080E06000000C0E03030E0C00A9
:10DDC00000E0E00000E0E00040474F68381F070037
:10DDD00000202020A0E06000000C0E0B09080800C5
:10DDE0001C14DCE02020E0C000000F1F10101C0CF1
:10DDF00000000000FF00000000000000FF00000025
:10DE00001C141CE0E02020200000001F1F01010066
:10DE100000060101020204040000000000000000EE
:10DE20000000F0F80868F8F00C00070F0B080F0767
:10DE30000000202030F8F8000C000000000F0F0058
:10DE4000000030380888F8700C000C0E0B09080828
:10DE5000000030388888F8700C00060E08080F079C
:10DE6000000000F8F800E0E00C00030302020F0FCE
:10DE70000000F8F8888888080C000808080C0703D8
:10DE80000000C0E07858C8800C00070F08080F0792
:10DE90000000080888E878180C00000E0F01000048
:10DEA000000070F8C888F8700C00070F08090F0709
:10DEB0000000F0F80808F8F00C0000090D0F03014D
:10DEC000000000E0F8180C0C0C8CCC78F8E0000096
:10DED0000000001F7F78CCC6C3C1C0607F1F000058
:10DEE00000000000303038FCFC00000000000000A2
:10DEF00000000000C0C0C0FFFFC0C0C000000000A4
:10DF000000000070781C0C0C0C0C8CDCF87000000D
:10DF1000000000C0E0F0F8DCCEC7C3C1C0C0000004
:10DF200000000070781C0C0C0C0C0C9CF8F000002D
:10DF30000000003878E0C3C3C3C3C3E77D380000E6
:10DF40000000000080C0E070381CFCFC00000000F5
:10DF50000000000F0F0D0C0C0C0CFFFF0C0C000050
:10DF6000000000FCFC8C8C8C8C8C8C8C0C0C0000CD
:10DF70000000003171E1C1C1C1C1C1E37F3E0000B9
:10DF800000000000C0E070381C0C0C0C0000000009
:10DF90000000003F7FE7C3C3C3C3C3E77E3C00006C
:10DFA0000000000C0C0C0C0C0C0CCCFC3C0C00000D
:10DFB000000000000000C0F03C0F03000000000063
:10DFC00000000000F0F89C0C0C0C9CF8F000000025
:10DFD0000000003C7EE7C3C3C3C3C3E77E3C000030
:10DFE000000000F0F89C0C0C0C0C0C9CF8F00000ED
:10DFF0000000000001C3C3C3E3733B1F0F03000015
:10E000000000000000000000000000000000000010
:10E010000000000000000000000000000000000000
:10E020000000000000000000F00000000000000000
:10E0300000000101010101011F01010101010100B5
:10E0400000000000000000000000000000000000D0
:10E0500000010101010101010101010101010100B2
:10E060000038283880C06060606060408000000038
:10E07000000000001F3F6060606060201000000032
:10E08000000000000000C0C0C0C000000000000090
:10E0900000000000000030303030000000000000C0
:10E0A0000038283800FCFC8C8C8C8C8C8C00000098
:10E0B00000000000007F7F0101010101010000005C
:10E0C000FCFC0000000000C0C00000000000FCFCE0
:10E0D0007F7F30180C0603010103060C18307F7F88
:10E0E000808040402020101008080404FE0000003A
:10E0F0000000010102020404080810103F000000A3
:10E100000000FE0404080810102020404080800019
:10E1100000003F1010080804040202010100000082
:10E12000008080C0C06060303018180C0CFE000009
:10E13000000101030306060C0C181830307F0000A4
:10E140000000FE0C0C181830306060C0C0808000E9
:10E1500000007F303018180C0C0606030301010084
:10E160008080C0C0E0E0F0F0F8F8FCFCFE000000A9
:10E1700000000101030307070F0F1F1F3F000000EE
:10E180000000FEFCFCF8F8F0F0E0E0C0C080800089
:10E1900000003F1F1F0F0F070703030101000000CE
:10E1A00080B500F005F9002094490968887200F0F4
:10E1B00045F99348002141604FF40441914A118090
:10E1C000016000209049086001BD10B500208F4912
:10E1D00088728F48C0798949096848720020FDF724
:10E1E000F3FB4FF400710020FDF7F5FB2021002028
:10E1F000FDF7FEFB18210020FDF77CFC854C94F810
:10E200002C100020FDF7AAFC58210020FDF764FC2B
:10E210000020FDF72FFC0020FDF71CFC0021012051
:10E22000FDF7D9FB98210120FDF756FC20210120A4
:10E23000FDF7DEFB00210120FDF7F3FB00210220AA
:10E24000FDF7C9FBD8210220FDF754FC94F82C10EF
:10E250000220FDF783FC4FF440510220FDF7E1FB63
:10E2600000210220FDF7C4FB94F82C100020FDF7DC
:10E2700075FC0020FDF7EEFB0020FFF795FA01206A
:10E280006149086064486549086000206449087075
:10E2900010BD5A480068807A002800D1704780B5C8
:10E2A0000520594908600120FDF704FC0220FDF714
:10E2B000EFFB00205A49087001BD584800685649D4
:10E2C000884202D00220FDF7EDBD704704204E4980
:10E2D000086070477047704780B548490A681378EE
:10E2E00003F07F03212B10D1FE280ED15088002887
:10E2F0000BD19088002808D1D088012805D10FF2D1
:10E300009D00030003D1022002BD022002BD9061E6
:10E3100000200968488200F041F8002002BD80B565
:10E32000364909680A7802F07F02212A17D1FF28AE
:10E3300015D14888002812D1888800280FD1C888B4
:10E3400000280CD10120FDF7B5FB0220FDF7A0FB52
:10E3500031483249086000203149087002BD02206E
:10E3600002BD002901D002207047002801D0022000
:10E370007047002070472B49FEF779BF2A49FEF706
:10E3800076BF1E490968C978062901DB002070475D
:10E39000264A02EBC101FEF76ABF0000002805D142
:10E3A00001201649096808820020704720487047FC
:10E3B000204A106851689268002800D1704710B454
:10E3C0001D4B98700446240A1C710446240C9C7151
:10E3D000000E187299720846000A18730846000C5D
:10E3E0009873090E19749A741046000A187510462D
:10E3F000000C9875120E1A7610BC7047A0330020DE
:10E40000405C0040683400205834002084330020F1
:10E4100024F500089C09002055534243583300203E
:10E4200078330020F0090020F8090020000A0020BD
:10E4300054340020E8F7FF1F480900200648012156
:10E4400001600021016041604FF4E051034A1180F6
:10E450000160002070470000405C004068340020EC
:10E4600001FF00E11FE000FF010000011E010001AB
:10E470001E010000006010109090E0000000000EEF
:10E48000111110081F1800001010F040201010305B
:10E49000000010101F1010000000000010F02010ED
:10E4A000101010E00000101F10000000101F1000DE
:10E4B00000001013F30000000000000010101F10F7
:10E4C0001000000010F02010101010E00000101FCD
:10E4D00010000000101F100000E010101010F010CD
:10E4E0000000007D8A8A8A8A917000000000008006
:10E4F000E0F8FE0707FEF8E080000000101C1F1F78
:10E500001F1F1F12121F1F1F1F1F1C10001C222164
:10E51000414141820700001E08101010100807003A
:10E5200000C0A090909090A0C000000708101010AC
:10E530001008040010F02010101010E00000101F50
:10E5400010000000101F100000202020202020209C
:10E5500020000000000000000000000001FF212159
:10E560002121F9030400101F1010101010180400CE
:10E57000001010F04020101030000010101F10107C
:10E5800000000000001010F04020101030000010BB
:10E59000101F10100000000001FF4140404041FFEB
:10E5A0000100101F10000000101F100000001013C9
:10E5B000F30000000000000010101F101000000009
:10E5C0000000E010101010F0100000609D8A8A8A90
:10E5D0008A91700001FF2010101010E00000101F41
:10E5E00010000000101F10000020202020202020FC
:10E5F00020000000000000000000000001077980FA
:10E60000008079070100000000071C0700000000DF
:10E6100000001010FE1010100000000000000F108D
:10E620001008000001FF0100000000000000101FA2
:10E63000101010101018040000C02010101010202E
:10E64000C0000007081010101008070010F000109C
:10E65000F01000F0100000031C0300031C03000076
:10E6600000202020202020202000000000000000AA
:10E670000000000001077980008079070100000098
:10E6800000071C070000000000C020101010102020
:10E69000C00000070810101010080700000010103C
:10E6A000FE1010100000000000000F101008000005
:10E6B00000806010080464940404B44C04848484CE
:10E6C0008484840404040404040484442464A4248A
:10E6D00024242424242424E404081060800000005E
:10E6E0000000806010080484C4E4E4E4E4C484040A
:10E6F00004040404040404040404040404040404DA
:10E70000040484C4E4E4E4E4C484081060800000E9
:10E7100000071820408082818082828585888F88CA
:10E7200088888F858585858585858D95A7B0AFA0DF
:10E73000A0A0A0A0A0A0A0BF8040201807000000BB
:10E7400000000718204080848C9C9C9C9F8F8783AE
:10E750008383838383838383838383838383838389
:10E760008383878F9F9C9C9C8C844020180700008B
:10E7700000806010080464940404B44C048484840D
:10E780008484840404040404040484442464A424C9
:10E7900024242424242424E404081060800000009D
:10E7A000000000F8F8808080F80080404040408001
:10E7B0000080404040408000004040F84040000061
:10E7C000D0004080404040800080404040800000B9
:10E7D00000071820408082818082828585888F880A
:10E7E00088888F858585858585858D95A7B0AFA01F
:10E7F000A0A0A0A0A0A0A0BF8040201807000000FB
:10E800000000001F1F0101011F000F121212120B46
:10E81000000C121212120F100000000F100800005E
:10E820001F00001F0000001F00478888887F00002D
:10E8300000E0F010102000008080808000008080C8
:10E84000F08080008080F0808000A00080008080C8
:10E8500080800000008080808000000000000000B8
:10E860000000806010080484C4E4E4E4E4C4840488
:10E870000404040404040404040404040404040458
:10E88000040484C4E4E4E4E4C48408106080000068
:10E89000000811111F0E000F121212120B000000BF
:10E8A0000F10080000000F1008001F00001F0000DC
:10E8B00000001F004F909090907F0000000000002B
:10E8C00000000718204080848C9C9C9C9F8F87832D
:10E8D0008383838383838383838383838383838308
:10E8E0008383878F9F9C9C9C8C844020180700000A
:10E8F000EB3C904D53444F53352E3000020108003D
:10E900000200025000F80C000100010000000000AD
:10E9100000000000000029A298E46C4E4F204E41F8
:10E920004D4520202020464154313220202033C93B
:10E930008ED1BCF07B8ED9B800208EC0FCBD007C8F
:10E94000384E247D248BC199E83C01721C83EB3A3C
:10E9500066A11C7C26663B07268A57FC750680CA82
:10E960000288560280C31073EB33C98A461098F7A9
:10E97000661603461C13561E03460E13D18B7611E2
:10E98000608946FC8956FEB82000F7E68B5E0B03D3
:10E99000C348F7F30146FC114EFE61BF0000E8E6F4
:10E9A00000723926382D741760B10BBEA17DF3A615
:10E9B0006174324E740983C7203BFB72E6EBDCA026
:10E9C000FB7DB47D8BF0AC9840740C487413B40E8E
:10E9D000BB0700CD10EBEFA0FD7DEBE6A0FC7DEBCF
:10E9E000E1CD16CD19268B551A52B001BB0000E8B7
:10E9F0003B0072E85B8A5624BE0B7C8BFCC746F05A
:10EA00003D7DC746F4297D8CD9894EF2894EF6C6E4
:10EA100006967DCBEA030000200FB6C8668B46F849
:10EA20006603461C668BD066C1EA10EB5E0FB6C863
:10EA30004A4A8A460D32E4F7E20346FC1356FEEBDF
:10EA40004A525006536A016A10918B4618969233C7
:10EA5000D2F7F691F7F64287CAF7761A8AF28AE871
:10EA6000C0CC020ACCB80102807E020E7504B4420A
:10EA70008BF48A5624CD136161720B4075014203F9
:10EA80005E0B497506F8C341BB000060666A00EB87
:10EA9000B04E544C44522020202020200D0A5265B4
:10EAA0006D6F7665206469736B73206F72206F746D
:10EAB000686572206D656469612EFF0D0A44697393
:10EAC0006B206572726F72FF0D0A5072657373204E
:10EAD000616E79206B657920746F20726573746143
:10EAE00072740D0A00000000000000ACCBD855AADB
:10EAF000F8B50020ADF80000604D4BF6BF7648F247
:10EB0000800729E055F82010ADF80010BDF800107E
:10EB100009040DD555F8201040F68F72114045F8C4
:10EB200020105748217800EB810050F8040C8047F2
:10EB3000BDF8000000060FD5207855F8201089B2E6
:10EB400048F60F72114045F820104E48217800EB2E
:10EB5000810050F8040C8047686C4B490880000421
:10EB600040F18B80088810F00F00484C2070C9D10C
:10EB7000474C28682080208800F030006080208882
:10EB800000F440502080286880B2304080F400506B
:10EB900080F02000384328600888C0062BD52868FC
:10EBA000ADF80000BDF80000000546D4BDF8000037
:10EBB0000004D1D5296840F68F7001402960FEF726
:10EBC000B9FD286880B206402088C00401D586F4CB
:10EBD00080562088800401D586F400566088C006DF
:10EBE00001D586F010066088800601D586F02006E3
:10EBF0003E432E60F1BD296889B248F60F7001408E
:10EC00002960FEF76EFD286880B206402088C004A7
:10EC100001D586F480562088800401D586F40056FC
:10EC20006088C00601D586F010066088800601D590
:10EC300086F020063E432E60F1BD296840F68F70B5
:10EC400001402960FEF71CFD286880B2064020883C
:10EC5000C00401D586F480562088800401D586F44E
:10EC600000566088C00601D586F0100660888006D0
:10EC700001D586F020063E432E60F1BD005C0040C9
:10EC800080090020640900206A34002072340020CA
:10EC90005034002000E010080810E00000000000E0
:10ECA000000F102020100F0000000000001010F8CE
:10ECB00000000000000000000020203F2020000095
:10ECC00000000000007008080888700000000000C4
:10ECD0000030282422213000000000000030088885
:10ECE00088483000000000000018202020110E008D
:10ECF000000000000000C02010F80000000000002C
:10ED000000070424243F24000000000000F80888C5
:10ED100088080800000000000019212020110E00C2
:10ED20000000000000E010888818000000000000CB
:10ED3000000F112020110E0000000000003808080C
:10ED4000C8380800000000000000003F000000007C
:10ED500000000000007088080888700000000000B3
:10ED6000001C222121221C000000000000E01008ED
:10ED70000810E000000000000000312222110F0006
:10ED80000000000000000000000000000000000083
:10ED900000303000000000000000000000E0180417
:10EDA00004040418E000000F3040404040300F00E1
:10EDB00000000808FC0000000000000040407F4008
:10EDC000400000000078040404040488700000601F
:10EDD0005048444241407000003804048484C830E4
:10EDE000000000384040404040211E00000080608C
:10EDF0001008FE0000000007040444447F4444005F
:10EE00000000FC0484848404040000384141404034
:10EE100040211E0000C03088848484041800000F44
:10EE20003140404040211E00001C04048444340C46
:10EE300004000000007E0100000000000070880453
:10EE4000040404887000001C2241414141221C003E
:10EE500000F0080404040418E0000030414242427B
:10EE60002219070000000000000000000000000060
:10EE700000000000000000001C1CC0300804040456
:10EE80000830000007182040404020101C120C02DF
:10EE900002FE8282E20200000000407F4000030088
:10EEA00080B53349086840F0010008604A6831487D
:10EEB00002404A600A68304802400A60086820F44C
:10EEC00080200860486820F4FE0048604FF41F006E
:10EED000886000F005F84FF000602849086001BD27
:10EEE00000222349086840F480300860086800F474
:10EEF0000030521C002802D1B2F5A06FF6D108688C
:10EF0000400C00F00100012830D11D48026842F099
:10EF1000100202600268920892000260026842F0E9
:10EF2000020202604868486048684860486840F4E7
:10EF300080604860486820F47C104860486840F46D
:10EF4000E8104860086840F0807008600868800138
:10EF5000FCD54868800880004860486840F002009E
:10EF60004860486800F00C000828FAD1704700009B
:10EF7000001002400000FFF8FFFFF6FE08ED00E081
:10EF8000002002400000000000000000000000001F
:10EF900000000000000000000000000080C0E0F061
:10EFA000F8FCFEFEFCF8F0E0C080C0E0F0F8FCFEEB
:10EFB000FEFEFC783080C0C000189CCEE6F0F8FC65
:10EFC000FEFEFCF8F0E0C0E0F0F87C00000000007D
:10EFD0000000000000000000000000000000000031
:10EFE0000000000000000000000000000000000021
:10EFF00000000000000000000000001F0F070301D8
:10F0000003070F1F3F7F7F3F1F0F07030103070702
:10F0100003191C0E6773391C0E07030103070F1F2A
:10F020003F7F7F3F1F0F070301000000000000002B
:10F0300000000000000000000000000000000000D0
:10F040000000000000003060C080000000000000F0
:10F05000000000000000180C060301000000000082
:10F060000000000000003060C0803060C080000000
:10F07000000000000000180C0603190C0603010034
:10F080000000000000003060C0803060C080306050
:10F09000C08000000000180C0603190C0603190CB0
:10F0A000060301000000183060C08000000000006E
:10F0B0000000000000000C0603010000000000003A
:10F0C000000000000000183060C0983060C0800070
:10F0D0000000000000000C0603010C060301000004
:10F0E000000000000000183060C0983060C0983008
:10F0F00060C0800000000C0603010C0603010C0632
:10F100000301000080B5F8F77FF84FF48040F8F76E
:10F11000B4F8F8F77FFAF8F7E6F8F8F7A1F9002065
:10F12000F8F77CFB0120F8F752F800F045F8FAF701
:10F130001EFFFAF72BFEF6F781FBF9F721F8F9F736
:10F14000FCFBF6F778FE1B48006B002805D01E215B
:10F1500041F28830F6F737FE03E000210846F6F763
:10F1600032FEFCF7D6FEFAF756FCF6F7EDFBF8F7A1
:10F170000CF8F4F7FCFFF6F794FC40F6B830F8F71B
:10F180004FFF4FF4AF7140F2DC50F8F708FBF8F78F
:10F190000BFA0120F8F728FCF7F7C8FCF7F7EDFCAD
:10F1A0004FF49670F7F7FFFFF8F750FFF6F79EFF62
:10F1B000FAE70000740000200448C06102210172D7
:10F1C00003490162034A4262086800478433002011
:10F1D0009C090020CC09002010188CC66363C68CE3
:10F1E0001810426331180C0C1831634200F01E1FD6
:10F1F000F00000FF8080FF0042C68C183030188C71
:10F20000C64208183163C6C6633118088C8CC6C65E
:10F210008C8CC6C68C8C31311818313118183131AC
:10F22000008C8C8C8C8C8C8C8C8C8C8C8C8C8C0036
:10F230000031313131313131313131313131310020
:10F2400080C0603098CC66333366CC983060C08024
:10F2500088CC6633190C060303060C193366CC8878
:10F26000113366CC983060C0C0603098CC663311E2
:10F270000103060C193366CCCC6633190C06030166
:10F28000F0B40246106895681318506803EB5004F8
:10F29000C0071CD54D441AE013F8017B05F8017B2B
:10F2A000491EF9D198B113F8011BC6F38106032E4C
:10F2B00008BF13F8016B01EB06214942801C294469
:10F2C00005D011F8016B05F8016B401EF9D1A3427E
:10F2D0000ED013F8016B16F0030104BF13F8011BE5
:10F2E000C91C30090F28DBD113F8010B0F30D7E709
:10F2F000F0BC02F10C00704700000010000010107C
:10F3000010101010001F1115111F0000111F100008
:10F31000001D1515151700151515151F000F0808E8
:10F320001F0800171515151D001F1515151D0001C7
:10F330000101011F001F1515151F00171515151FB9
:10F34000000708100807000000000000000F100E62
:10F35000100F000070B50E4C0E4D286820800E4E28
:10F36000218830880140480505D50C484068804711
:10F370004FF6FF302860218830880140080406D508
:10F38000FFF7B6FB0120BDE87040F6F7EAB970BDA3
:10F390006A340020445C0040683400209C0900204E
:10F3A000FCF71ABCFCF743BC7047FEE7FEE7FEE73C
:10F3B000FEE77047704770477047FFF7CBBFF8F71D
:10F3C0005CB9F8F7A2B980B54FF40070FCF747FFBD
:10F3D000002807D04FF40070FCF74DFFBDE8014056
:10F3E000FAF79FB901BD0000312E33300000000054
:10F3F0000000000000000000D0070000B80B000073
:10F4000064000000504600001200000000000000F0
:10F410000000000082000000010000000000000069
:10F42000202020202328303A53686F7720766F6C95
:10F43000746167652C313A53686F7720706F776518
:10F4400072290D0A000000002603530054004D00ED
:10F450006900630072006F0065006C006500630066
:10F46000740072006F006E0069006300730000009A
:10F470002603530054004D003300320020004D009D
:10F480006100730073002000530074006F0072006D
:10F49000610067006500000010B507497944183124
:10F4A000064C7C44163404E00A68081D1144884761
:10F4B0000146A142F8D110BD2C0000004800000018
:10F4C00000800202200000004D696E692044534F05
:10F4D0004469736B20202020202020202020202021
:10F4E000202020203384FFFFCC290000A80A002020
:10F4F000000000008DFDFFFF9C0300001A070000C4
:10F5000000000020202020202328433A3130307E84
:10F510003430302C463A3231327E373532290D0ABA
:10F520000000000009022000010100C032090400AF
:10F53000000208065004070581024000000705028A
:10F540000240000000F00DF8002801D0FFF7A4FFF2
:10F55000AFF300800020AFF30080FFF7D3FD00F091
:10F5600002F80120704700F001B800000746384655
:10F57000FDF700FDFBE700002020202328433A315F
:10F5800030307E3430302C463A3231327E373532AC
:10F59000290D0A0020202020202020202328303A76
:10F5A0004C6566742C313A5269676874290D0A00FB
:10F5B00020202020202020202328303A432C313ABC
:10F5C00046290D0A000000002020202020202328AA
:10F5D000303A4F46462C313A4F4E290D0A00000072
:10F5E00012010002000000408304205700020102C3
:10F5F00003010000202020232836307E39393929A4
:10F600000D0A000020202020232831367E323429A4
:10F610000D0A0000202020202328317E3235290DBC
:10F620000A00000020202023283130307E31343081
:10F63000290D0A0010035300540020004D00610002
:10F64000730073000148804701480047A1EE00089D
:10F65000C1F6000853686F775479706500000000A8
:10F6600053746254656D703D32303000576B546591
:10F670006D703D3330300000536C7054696D653DE2
:10F680003138300052617465645F503D313800009C
:10F6900054656D705374703D313000004F6666568E
:10F6A0006F6C743D313330004C6F774375723D3170
:10F6B0000000000053686F77547970653D3000009A
:10F6C000AFF30080AFF30080FFF73CFF5374625448
:10F6D000656D7000576B54656D700000536C70540D
:10F6E000696D650052617465645F500054656D70AA
:10F6F000537470004F6666566F6C740054656D707D
:10F700000000000048616E64000000004C6F774309
:10F710007572000054656D703D30000048616E6484
:10F720003D300000576B54656D7020005374625477
:10F73000656D7000536C7054696D6500506F77652E
:10F740007220200054656D70537470004F666656C9
:10F750006F6C740054656D702020200048616E64E9
:10F76000202020004C6F7743757220005368775437
:10F7700079706500686A6C747A4C000004030904AF
:10F78000FFF712BEFFF711BEFFF710BEFFF70FBE67
:10F79000FFF70EBEFFF70DBEFFF70CBEFFF70BBE67
:10F7A000FFF70ABEFFF7FEBFFFF7FEBFFFF7FEBF82
:10F7B000FFF7FEBFFFF7FEBFFFF7FEBFFFF7FEBF7D
:10F7C000FFF7FEBFFFF7FEBFFFF7FEBFFFF7FEBF6D
:10F7D000FFF7FEBFFFF7FEBFFFF7FEBFFFF7FEBF5D
:10F7E000FFF7FEBFFFF7FEBFFFF7FEBFF7F7FCBF57
:10F7F000FFF7FEBFFFF7E1BDFFF7FEBFFFF7FEBF5C
:10F80000FFF7E1BDFFF7FEBFFFF7FEBFFFF7FEBF4B
:10F81000FFF7FEBFFFF7D3BDFFF7D3BDFFF7FEBF76
:10F82000FFF7FEBFFFF7FEBFFFF7FEBFFFF7FEBF0C
:10F83000FFF7FEBFFFF7FEBFFFF7FEBFFFF7FEBFFC
:10F84000FFF7FEBFFFF7FEBFFFF7FEBFFFF7FEBFEC
:10F85000FFF7FEBFFFF7FEBFFFF7FEBFFFF7FEBFDC
:10F86000FFF7FEBFFFF7FEBFFFF7FEBFFFF7FEBFCC
:10F87000FFF7FEBFFFF7FEBFFFF7FEBFFFF7FEBFBC
:10F88000FFF7FEBFFFF7FEBFFFF7FEBFFFF7FEBFAC
:10F89000FFF7FEBFF2200001F0012A803F0001F3D4
:10F8A00041330001100378F50008040422F4081025
:10F8B00002F60008140412240412B0101294041268
:10F8C000C804100720F40008A8320020C804100360
:10F8D000A83000206020126C0412780412840412F4
:10F8E0009004229C3C1002F700081C0412A80C1281
:10F8F000B404F2FF0001F1F2011ACC1812D4041280
:10F90000DC0412E40412EC0412F40412FC041A04E1
:10F910003C120C049A543C00FE88130000560E4B17
:10F920000E410E360E2B0E1F0E140E080EFD0DF09E
:10F930000DE40DD80DCB0DBE0DB10DA40D960D89A6
:10F940000D7B0D6D0D5E0D500D410D320D230D140F
:10F950000D040DF50CE50CD50CC40CB40CA30C92E5
:10F960000C810C700C5F0C4D0C3B0C290C170C041B
:10F970000CF20BDF0BCD0BB90B8E0F930B800B6CC6
:10F980000B580B440B300B1C0B080BF30ADF0ACA95
:10F990000AB60AA10A8C0A770A620A4C0A1F0E22CA
:10F9A0000A0C0AF709E109CC09B609A0098B097507
:10F9B000095F09490933091D090809F208DC08C66D
:10F9C00008B0089A0885086F08590843082E0818D7
:10F9D000080308ED07D807C207AD07980783076E2D
:10F9E00007580744072F071A070507F106DD06C861
:10F9F00006B406A0068C067806650651063E062B60
:10FA00000617060406F205DF05CC05BA05A805961B
:10FA1000058305720560054F05144B3D052C051B3C
:10FA2000050A05F904E904D804C804B804A8049830
:10FA300004890479046A045B044C043D042F042007
:10FA40000412040404F603E803DB03CD03C003B38C
:10FA500003A60399038C038003740367035B034FBE
:10FA6000034403380300000155566A59123C08103C
:10FA70001AAED552A80FC0D30040A08D14DA02816F
:10FA800033D9F1DB30A4A6AF00040C74801F200230
:10FA900080740C042E4003031C601C033713804049
:10FAA00001211C100300001F22420116229F300377
:10FAB00000004040C01B12C00D7C0440407F41400C
:10FAC00040FB038F60600604710C237804012388D7
:10FAD000780FEC0660504844424140702D04A13933
:10FAE0001001E018083210010818E01310010F305F
:10FAF000206A300120300F1F70010808FC27117A9E
:10FB000092407AF1FF01F105011E247003122C04CA
:10FB1000123404123C041244042E4C8403110412C7
:10FB20005C04126404126C0443CA7904A55FF3FFF9
:10FB3000100001F19501A5B81EA048031EE8DE03E0
:10FB4000C364000C400C3C86010070170000B80B29
:10FB500000001800342D400412FA04520A04438CA9
:10FB6000002C5201042101F1170C4004601D00001B
:10FB70004808401C051A03530054004DE008A00437
:10FB800032003100300001F00409A1F300082DD843
:10FB900004F206A5201003A1E10008CB041003D550
:10FBA000E20008D70412D90410031FE3000863041D
:10FBB000127704127D044B83E3D02D34042134C327
:10FBC00093E24492BB1012CD0C1EE00C0912122CD1
:10FBD0002E24140911081E7C18032D22051E48200E
:10FBE000091226085270081003480900201A081E3E
:10FBF00034C80625383D3D054206D75DE804C30AF2
:10FC000000013188120205F00207BE80000804528C
:10FC1000FF01F20056141139D30101535603730248
:01FC20000AD9
:040000050800F6C138
:00000001FF
